:10686500EF24FEFFEE34FFFEE48F488E47F546F534
:10687500459056D8E0FFE4FCFDFEAB48AA47A94683
:10688500A8451240B48F488E478D468C459056F6E4
:10689500E0FCA3E0FDA3E0FEA3E02548F548EE35C6
:1068A50047F547ED3546F546EC3545F545AF48AE78
:0468B50047AD46FCA9
:0168B90022BC
:106969009056D6E0C313FCA3E013FD12405FAB07BA
:10697900AA069056EEA3A3E0FEA3E02BFBEE3AFE97
:02698900AF035A
:01698B0022E9
:1069F8009056D6E0C313FCA3E013FD12405FED25CB
:066A0800E0FFEC33FE226A
:0463C4008E458F462D
:1063C8001269698E478F48AF46AE451269F88E4903
:1063D8008F4AAE47AF48E4FCFD90401CE0F8A3E0CC
:1063E800F9A3E0FAA3E0FBC31241D1602BAE47AF9B
:1063F80048E4FCFD755B01755C01755D77755E0BA6
:106408001268F5EF70057EFF7FFF22AE47AF48E4C4
:10641800FCFD90401C12423D740C254AF5827477AD
:106428003549F583E0754500F546754600F5457430
:106438000B254AF58274773549F583E02546F546FC
:08644800E43545F545FEAF46C1
:016450002229
:085E78008F368E358D348C331A
:105E80009056D8E0FF7E009056D6E0FCA3E0FD12CD
:105E9000404D8E378F38904005E0FCA3E0FDA3E035
:105EA000FEA3E0FF90400D12423DAE37AF38E4FC58
:105EB000FDAB36AA35A934A833D31241D14051AE37
:105EC00037AF38AB07AA06E5369BF536E5359AF5C8
:105ED00035E5349400F534E5339400F53390400D06
:105EE000A3A3E0FEA3E0FF1263C4E4FCFD90400D19
:105EF00012423DE47FFF7EFFFDFC90400DE0F8A3E1
:105F0000E0F9A3E0FAA3E0FBC31241D1709CFF22A9
:105F10009056D6E0FEA3E0FBAA06E4F9F8AF36AE51
:105F200035AD34AC3312413F904017EFF090400D47
:105F3000A3A3E0FEA3E0FF126865A804A905AA06D2
:105F4000AB07904017E0FFE4FCFDFEEB2FFFEE3ABD
:105F5000FEED39FDEC38FC90401112423D9056D6D2
:105F6000E0FEA3E0FBAA06E4F9F8AF36AE35AD34A7
:105F7000AC3312413FAF03904015EAF0A3EFF0902D
:0B5F8000401C124249000000007F019D
:015F8B0022F3
:045F8C008E3A8F3B7F
:105F9000D3E53B9401E53A94005003026097E53B5A
:105FA00094F0E53A94FF4003026097AF3BAE3A129B
:105FB00069698E3C8F3DAF3BAE3A1269F88E3E8FD9
:105FC0003FAE3CAF3DE4FCFD755B01755C01755D6A
:105FD00057755E0B1268F5EF6057AE3AAF3BE4FCC5
:105FE000FD905706E0F8A3E0F9A3E0FAA3E0FBD3A5
:105FF0001241D1400DAE3AAF3BE4FCFD9057061282
:10600000423D740C253FF5827457353EF583E075AB
:106010003A00F53B753B00F53A740B253FF5827469
:1060200057353EF583E0253BF53BE4353AF53A80BC
:10603000037F0022740B253FF5827457353EF583AC
:10604000E4F0740C253FF5827457353EF583E4F097
:10605000F5409056D9E0FFE540C39F4003025F90B2
:106060007F05126A68AF407E009056E0E0FCA3E036
:10607000FD12404DE53D2FFFE53C3EFEE4FCFD7585
:106080005B01755C01755D57755E0B12692FEF70D2
:0960900002FF22054080BB7F01E4
:0160990022E4
:104F3100E4F54EF54F905706A3A3E0FEA3E0FF1260
:104F41006969E48F558E54F553F5529056EEE0F8A9
:104F5100A3E0F9A3E0FAA3E0FBC3E5559BFFE55409
:104F61009AFEE55399FDE55298FCA804A905AA0605
:104F7100AB079056D6E0C313FEA3E013FFE4FCFD9C
:104F81001240B48E4E8F4F9056E0E0FEA3E0FFE456
:104F9100FCFD9056EEE0F8A3E0F9A3E0FAA3E02FC0
:104FA100FFEA3EFEED39FDEC38FCAB55AA54A9539E
:104FB100A852C31241D14003025119AF55AE54ADAD
:104FC10053AC52755B01755C01755D57755E0B12D3
:104FD10068F5EF7003FEFF22E4F550F551D39056CA
:104FE100D7E095519056D6E0955050030250E974A0
:104FF1000B2551F58274573550F583E0600302505B
:10500100DB740C2551F58274573550F583E060034C
:105011000250DB740B2551F58274573550F58374BA
:10502100FFF0740C2551F58274573550F58374FFE8
:10503100F0E4F5569056D9E0FFE556C39F503D7F09
:1050410005126A68AF567E009056E0E0FCA3E0FDD1
:1050510012404DEF2555FFEE3554FEE43553FDE486
:105061003552FC755B01755C01755D57755E0B1200
:10507100692FEF7003FEFF22055680B8E550C31378
:10508100FEE55113254FF54FEE354EF54EE54F2414
:10509100FEFFE54E34FFFEE4FCFD905702E0F8A36D
:1050A100E0F9A3E0FAA3E0FBD31241D1406AAE4E8E
:1050B100AF4FE4FCFD905706E0F8A3E0F9A3E0FA56
:1050C100A3E0FB1241D1500DAE4EAF4FE4FCFD9079
:1050D100570612423DAE4EAF4F2274022551F55193
:1050E100E43550F550024FDE9056D6E0C313FEA3CF
:1050F100E013254FF54FEE354EF54EE5552401F5FC
:1051010055E43554F554E43553F553E43552F5522D
:0B5111007F01126A68024F88E4FEFF75
:01511C002270
:046262008E458F4690
:10626600124F318E478F48E54845477003FEFF229F
:10627600AF46AE451269698E498F4AAF46AE4512A2
:1062860069F88E4B8F4CAE49AF4AE4FCFD755B0155
:10629600755C01755D57755E0B1268F5EF60667487
:1062A6000B254CF5827457354BF583E548F0E547E9
:1062B600FF740C254CF5827457354BF583EFF0E4EB
:1062C600F54D9056D9E0FFE54DC39F503C7F051232
:1062D6006A68AF4D7E009056E0E0FCA3E0FD1240F8
:1062E6004DE54A2FFFE5493EFEE4FCFD755B017571
:1062F6005C01755D57755E0B12692FEF7003FEFF2B
:0D63060022054D80BDE4FEFF22AE47AF48EA
:016313002267
:0669AE0014F9123FD3FFB3
:1069B4007E08C2B4EF3392B3EF25E0FFD2B4DEF227
:0269C400D2B34C
:0169C60022AE
:0669C70014F9EF12401963
:1069CD007E08C2B4D2B4EF25E0FF30B50343070112
:0269DD00DEF0EA
:0169DF002295
:106A0E00E4FC1269CDAD07ED6009ED640160040C84
:056A1E00BC09EFAF050B
:016A23002250
:10000300EF4440FF1269B4AF671269B4AF68126975
:10001300B4AF691269B4AF6A1269B4AF6B0269B461
:10674100E4F52FF530F531F5327D01D2B2FC7FFF52
:106751001269B40CBC0AF7C2B2E4F56AF569F568CE
:10676100F567756B95FF120003126A0EAD07ED64B4
:106771000160037F0022BD0124D2B27FFF1269B400
:10678100C2B2756A007569C07568FF756700756B7F
:10679100FF7F01120003126A0EAD0780D9D2B27FCA
:0667A100FF1269B47F0144
:0167A70022CF
:0E6314008B5F8A6089618F658E648D638C62F9
:10632200C2B28F6A8E698D688C67756BFF7F181297
:106332000003126A0EEF60030263C17FFF1269B4A9
:106342007FFF1269B47FFF1269B47FFE1269B4E461
:10635200FDAB5F0561E561AA60700205601269AE7E
:10636200AB5F0561E561AA60700205601269AEABC0
:106372005F0561E561AA60700205601269AEAB5FFC
:106382000561E561AA60700205601269AE0DBD800B
:10639200C07FFF1269B47FFF1269B41269CDAD07E5
:1063A2001269CDEF60FA53050FD2B27FFF1269B4C2
:1063B200BD0B037F0022BD05037F01227F00227FE8
:0163C20000DA
:0163C30022B7
:0E64DC008B5F8A6089618F658E648D638C6230
:1064EA00C2B28F6A8E698D688C67756BFF7F1112D5
:1064FA000003126A0EEF705C1269CDBFFEFAE4FD6A
:10650A001269CDAB5F0561E561AA60700205601290
:10651A0069C7AB5F0561E561AA607002056012692F
:10652A00C7AB5F0561E561AA60700205601269C7C1
:10653A00AB5F0561E561AA607002056014F9EF12AC
:10654A0040190DBD80BA1269CD1269CDD2B2126955
:06655A00CD7F01227F004D
:016560002218
:086A60008F993099FDC29922C3
:036A68008F572223
:026A3800AB07AA
:0C6A3A00EDFEEBFF907913EEF0A3EFF0FF
:016A4600222D
:086561008F588E578D568C55A2
:10656900AF60AE5FAD5EAC5D78101241F5E4FFFE41
:10657900E4FCC004C005C006C007AF64AE63AD62E9
:10658900AC6178181241F5D003D002D001D000EBEC
:10659900FFEAFEE9FDEC48FCC004C005C006C007DF
:1065A900AF5CAE5BAD5AAC5978081241F5D003D057
:1065B90002D001D000EA4EFAE558FFEB4FFFEAFEA0
:1065C900E9FDE8FC90791612423D907916E0FCA3AA
:0865D900E0FDA3E0FEA3E0FFDA
:0165E1002297
:0D6A47007580FF7590FF75A0FF75B0FF22F0
:1069E00075985343878075C83075CBFF75CAF4C25C
:0869F00099C298D2CAD2AC2270
:105D6200126A471269E0E4F52890000012424900E5
:105D7200000000907930124249000000007F4090FC
:105D8200570BE4F0A3DFFCD2AF90790FE0FCA3E065
:105D9200FDA3E0FEA3E02401FFE43EFEE43DFDE4BA
:105DA2003CFC90790F12423DE47FE87E03FDFC90BB
:105DB200790FE0F8A3E0F9A3E0FAA3E0FBD31241E4
:105DC200D1402BC2AF90790F12424900000000D29D
:105DD200AF126741EF600CE5247013752201752440
:105DE20001800BE524B40106752101E4F524E522C6
:105DF2006037C2AFE4F522752301900000124249D8
:105E020000000000907930124249000000009040EA
:105E12001C1242490000000090570612424900003D
:105E22000000C290752901D2AFE521600FC2AFE434
:105E3200F521F523F520D290D291D2AFE528601555
:105E4200C2AFE4F52890570AE06005125B23800395
:105E52001259FCD2AFE5297003025D8BC2AFE4F5A3
:105E62002912284FEF6007752001C2918003E4F5E3
:065E720020D2AF025D8B9F
:030023000254A1E3
:1054A100C0E0C0F0C083C082C0D075D000C000C0D1
:0D54B10001C002C003C004C005C006C00752
:1054BE00752A01752B56752CA4C292209805D2928E
:1054CE000255FA752D00752E0090790B1242490087
:1054DE0000000020981390790B124208E47B257A85
:1054EE004EF9F8D31241D150EAE47F207E4EFDFCF6
:1054FE0090790BE0F8A3E0F9A3E0FAA3E0FBD31256
:10550E0041D140030255D0AB2AAA2BA92C852E825D
:10551E00852D83E59912402BC298052EE52E70023B
:10552E00052D6425452D70A19056A4E0FF640460FE
:10553E000DEF64056008EF640960030255F3E4FFA4
:10554E007E08FDFC9056A5E0F8A3E0F9A3E0FAA3CF
:10555E00E0FBD31241D1400E9056A474FFF0752893
:10556E0001D2920255FA752D00752E00AE2DAF2E7A
:10557E00E4FCFD9056A5E0F8A3E0F9A3E0FAA3E061
:10558E00FBD31241D1405E90790B124249000000CC
:10559E000020981390790B124208E47B257A4EF97D
:1055AE00F8D31241D150EAE47F207E4EFDFC907973
:1055BE000BE0F8A3E0F9A3E0FAA3E0FBD31241D18C
:1055CE0040089056A474FFF0801B7402252EF582BD
:1055DE007400352DF583E599F0C298052EE52E70F1
:0C55EE008B052D8087752801C298D29291
:1055FA00D007D006D005D004D003D002D001D00005
:0B560A00D0D0D082D083D0F0D0E032AE
:106451007531017532567533C9C293E4F52FF530A4
:10646100AB31AA32A933853082852F83123FECFFED
:10647100126A600530E5307002052FC39405E52FDF
:10648100940040DCE4FFFEFDFC9056CAE0F8A3E076
:10649100F9A3E0FAA3E0FBC31241D1603BE4F52F7D
:1064A100F530AE2FAF30E4FCFD9056CAE0F8A3E022
:1064B100F9A3E0FAA3E0FBD31241D1401B740225FA
:1064C10030F5827400352FF583E0FF126A600530E4
:0A64D100E53070CE052F80CAD2938B
:0164DB00229E
:1059FC00E49056C9F0A3124249000000009056A44E
:105A0C00E0B40D004003025B1D905A1CF82828736B
:105A1C00025A43025A48025A4D025A67025A7002FD
:105A2C005AA5025ABE025ACE025AD3025ADF025B60
:105A3C000B025B10025B151222F6805A1236518053
:105A4C00559056A5E0FCA3E0FDA3E0FEA3E0FF7B90
:105A5C00017A007902124538025B189056A512663D
:105A6C005F025B181236519056C9EFF060089040F7
:105A7C000912665F80209056A5E0FCA3E0FDA3E030
:105A8C00FEA3E0FF7536017537007538027B017A8D
:105A9C005679A91208A4025B189056A5E0FCA3E065
:105AAC00FDA3E0FEA3E0FF7B017A00790212172C24
:105ABC00805AE4904004F07B017A5679A912328E18
:105ACC00804A1258D18045E52060469056C9740131
:105ADC00F0803E124CC59056C9EFF070349056A52C
:105AEC00E0FCA3E0FDA3E0FEA3E0FF7536017537F3
:105AFC00007538027B017A5679A9120026800D12A6
:105B0C004CC580081265E28003126A249056C9EFD6
:075B1C00F01264517F012229
:1022F600E5207002FF22E4F52FF530F534F536F5CA
:1023060031F53290402075F020E53212427AE531FF
:1023160075F020A425832532F583E4F090402175DD
:10232600F020E53212427AE53175F020A42583F8D3
:102336002532F583E4F00532E53270020531641486
:10234600453170BF900000E07002A3E060030225F3
:10235600B7F535D39056DBE095359056DAE0940024
:1023660050030225A7E4FCFDFE9056F2E0F8A3E038
:10237600F9A3E0FAA3E02535FFEE3AFEED39FDECD0
:1023860038FC755B01755C01755D57755E0B1268EF
:10239600F5EF7002FF22E4F531F532D39056D7E01F
:1023A60095329056D6E09531500302259C740B2544
:1023B60032F58274573531F583E0FF70028057EFAE
:1023C60064E5700302258EE4F533E533FD7C0025D4
:1023D60032FFEC3531FE740B2FF58274573EF583D0
:1023E600E0FBE530AE2F7805C333CE33CED8F92DDA
:1023F600FFEE3CFE74022FF58274003EF583EBF08F
:102406000533E533B420C30530E5307002052FC32C
:10241600E52F9402400675340102259CE536C394E7
:1024260014400302258E74162532F5827457353111
:10243600F583E0640F600302254A740B2532F582AA
:1024460074573531F583E0541F1475F01AA4F53826
:10245600D394E0400302258EE4F5377533017E0000
:10246600E5322533FFEE3531FE740B2FF5827457B6
:102476003EF583E0FFE537FDE5382DFDE433FC75D9
:10248600F020E536A42420F582E5F03440F58325D6
:1024960036F583E5822DF582E5833CF583EFF0057D
:1024A600370533E533B40BB675330E7E00E53225BA
:1024B60033FFEE3531FE740B2FF58274573EF583EC
:1024C600E0FFE537FDE5382DFDE433FC75F020E54A
:1024D60036A42420F582E5F03440F5832536F583CD
:1024E600E5822DF582E5833CF583EFF0053705336C
:1024F600E533B41AB675331C7E00E5322533FFEE9C
:102506003531FE740B2FF58274573EF583E0FFE5F7
:1025160037FDE5382DFDE433FC75F020E536A424BF
:1025260020F582E5F03440F5832536F583E5822DE6
:10253600F582E5833CF583EFF005370533E533B4E3
:1025460020B68044E4F5337E00E5322533FFEE35D0
:1025560031FE740B2FF58274573EF583E0FF75F05C
:1025660020E536A42420F582E5F03441F5832536AE
:10257600F583E5822533F582E43583F583EFF005AF
:1025860033E533B420C1053674202532F532E435FF
:1025960031F5310223A1E5346401600505350223D6
:1025A60059E530AE2F7805C333CE33CED8F902289D
:1025B60042900000E0FFA3E0904002CFF0A3EFF0CE
:1025C600904002E0FEA3E0FF1268659056A012421A
:1025D6003DE4F5359056D8E0FFE535C39F4003024C
:1025E6002811E4FCFDFE9056A0E0F8A3E0F9A3E074
:1025F600FAA3E02535FFEE3AFEED39FDEC38FC7521
:102606005B01755C01755D57755E0B1268F5EF70C1
:1026160002FF22E4F531F532D39056D7E095329099
:1026260056D6E095315003022806740B2532F58202
:1026360074573531F583E0FF7006753401022806BC
:10264600EF64E570030227F8E4F533E533FD7C001B
:102656002532FFEC3531FE740B2FF58274573EF5AB
:1026660083E0FBE530AE2F7805C333CE33CED8F901
:102676002DFFEE3CFE74022FF58274003EF583EBCF
:10268600F00533E533B420C30530E5307002052F7D
:1026960074162532F58274573531F583E0640F6080
:1026A600030227B4740B2532F58274573531F5834E
:1026B600E0541F1475F01AA4F538D394E0400302D1
:1026C60027F8E4F5377533017E00E5322533FFEE52
:1026D6003531FE740B2FF58274573EF583E0FFE526
:1026E60037FDE5382DFDE433FC75F020E536A424EE
:1026F60020F582E5F03440F5832536F583E5822D15
:10270600F582E5833CF583EFF005370533E533B411
:102716000BB675330E7E00E5322533FFEE3531FEFE
:10272600740B2FF58274573EF583E0FFE537FDE520
:10273600382DFDE433FC75F020E536A42420F5821F
:10274600E5F03440F5832536F583E5822DF582E5FF
:10275600833CF583EFF005370533E533B41AB675D8
:10276600331C7E00E5322533FFEE3531FE740B2F28
:10277600F58274573EF583E0FFE537FDE5382DFD1C
:10278600E433FC75F020E536A42420F582E5F03428
:1027960040F5832536F583E5822DF582E5833CF504
:1027A60083EFF005370533E533B420B68044E4F50E
:1027B600337E00E5322533FFEE3531FE740B2FF5FF
:1027C6008274573EF583E0FF75F020E536A4242099
:1027D600F582E5F03441F5832536F583E582253328
:1027E600F582E43583F583EFF00533E533B420C194
:1027F600053674202532F532E43531F53102261ED0
:10280600E5346401600505350225DAE534640160C6
:102816001E904002E0FEA3E0FF1263C4904002EE69
:10282600F0A3EFF0D394EFEE94FF50030225C6E534
:1028360030AE2F7805C333CE33CED8F9FFE4FCFD96
:082846009056CA12423D7F01C9
:01284E002267
:063651007B017A5679A905
:063657008B2F8A3089313F
:10365D00E5207002FF22E4904004F0900000E0703D
:10366D0002A3E0600302378FF536D39056DBE09569
:10367D00369056DAE09400500302377AE4FCFDFEF2
:10368D009056F2E0F8A3E0F9A3E0FAA3E02536FFA7
:10369D00EE3AFEED39FDEC38FC755B01755C01759C
:1036AD005D57755E0B1268F5EF7002FF22E4F5327F
:1036BD00F533D39056D7E095339056D6E0953250EA
:1036CD000302376F740B2533F58274573532F5834A
:1036DD00E07002FF22E4F534AB2FAA30A931853416
:1036ED0082758300123FECFFE5347C002533FDEC41
:1036FD003532FC740B2DF58274573CF583E0B5071C
:10370D00090534E534D3940A40CEE534D3940A4008
:10371D004374162533F58274573532F583E020E472
:10372D0033E4F5347E00E5332534FFEE3532FE7497
:10373D000B2FF58274573EF583E0FF74022534F5A7
:10374D0082E43400F583EFF00534E534B420D5750B
:10375D003501800E74202533F533E43532F5320210
:10376D0036BFE535640160050536023677D39056D0
:10377D00DBE095369056DAE0940040030238E77F9F
:10378D000022900000E0FFA3E0904002CFF0A3EFF5
:10379D00F0904002E0FEA3E0FF1268659056A01283
:1037AD00423DE4F5369056D8E0FFE536C39F400321
:1037BD000238B1E4FCFDFE9056A0E0F8A3E0F9A3B9
:1037CD00E0FAA3E02536FFEE3AFEED39FDEC38FCCC
:1037DD00755B01755C01755D57755E0B1268F5EFD4
:1037ED007002FF22E4F532F533D39056D7E09533CE
:1037FD009056D6E0953250030238A6740B2533F55A
:10380D008274573532F583E07002FF22E4F534AB54
:10381D002FAA30A931853482758300123FECFFE564
:10382D00347C002533FDEC3532FC740B2DF58274A0
:10383D00573CF583E0B507090534E534D3940A40C8
:10384D00CEE534D3940A404374162533F58274576C
:10385D003532F583E020E433E4F5347E00E533259D
:10386D0034FFEE3532FE740B2FF58274573EF5831F
:10387D00E0FF74022534F582E43400F583EFF005A2
:10388D0034E534B420D5753501800E74202533F51B
:10389D0033E43532F5320237F6E53564016005055E
:1038AD00360237B2E5356401601E904002E0FEA39A
:1038BD00E0FF1263C4904002EEF0A3EFF0D394EF5B
:1038CD00EE94FF500302379ED3904003E094EF90A7
:1038DD004002E094FF40037F00229040047401F009
:1038ED0090001CE0FF7E00A3E0FD7C00126A38E42E
:1038FD00FCFD90400512423D90001EE0FFE4FCFDF2
:10390D00FEC007A3E0FFE48F5CF55BF55AF559A304
:10391D00E0FFE48F60F55FF55EF55DA3E0FFE48FFA
:10392D0064F563F562F561D0071265619040091287
:10393D00423D904005E0FCA3E0FDA3E0FEA3E0FFC7
:10394D0090400D12423D904005A3A3E0FEA3E0FF81
:10395D0012686590401112423DE4904015F0A3F0BD
:10396D00A3F090401C124249000000009040181234
:10397D004249000000009056CA1242490000002042
:02398D007F01B8
:01398F002215
:0E4538008F328E318D308C2F8B338A34893543
:10454600E5207002FF22904004E07002FF228532CF
:104556003D85313C85303B852F3AE4F538F539FF0A
:104566007E40FDFCAB32AA31A930A82FD31241D12F
:1045760040037F0022904018E0FCA3E0FDA3E0FE8C
:10458600A3E02532FFEE3531FEED3530FDEC352F5B
:10459600FC904009E0F8A3E0F9A3E0FAA3E0FBC32E
:1045A6001241D150037F0022E4FFFEFDFCAB32AA8C
:1045B60031A930A82FD31241D150030247A290400F
:1045C60015E0FEA3E0FFEF2532FBEE3531FAE435C8
:1045D60030F9E4352FF89056D6E0FEA3E0FFE4FC70
:1045E600FDD31241D1400C9056D6E0F536A3E0F546
:1045F600378010904016E02532F537904015E035AB
:1046060031F536D3904016E09400904015E09400C2
:104616005003024698904011E0FCA3E0FDA3E0FEA3
:10462600A3E0FF755B01755C01755D57755E0B1246
:1046360068F5EF605A904015E0FEA3E0FFC3E5374A
:104646009FF537E5369EF536E4FFFEC3EF9537EE68
:104656009536502B904016E02FFD904015E03EFC1D
:10466600740B2DF58274573CF583E0AB33AA34A95D
:10467600358F828E8312402B0FBF00010E80CC90A7
:104686004016E02537F0904015E03536F080367F4D
:104696000022904011E0FCA3E0FDA3E0FEA3E0FFB2
:1046A600755B01E5352539F9E534353885335CF533
:1046B6005D895E1268F5EF7002FF22904015E536BF
:1046C600F0A3E537F0AE36AF37AB07AA06C3E5323F
:1046D6009BF532E5319AF531E5309400F530E52F5A
:1046E6009400F52FE5372539F539E5363538F538AF
:1046F6009056D7E024FFFF9056D6E034FFFE904058
:1047060015E0FCA3E0FDD39FEC9E50030245AE905E
:1047160056D6E0FEA3E0FFED9FFFEC9E904015F01D
:10472600A3EFF0A3E004F09056D8E014FF904017F2
:10473600E0D39F4045E4F090400DA3A3E0FEA3E044
:10474600FF1263C4E4FCFD90400D12423DE47FEF8E
:104756007EFFFDFC90400DE0F8A3E0F9A3E0FAA38C
:10476600E0FBD31241D140037F002290400DA3A36A
:10477600E0FEA3E0FF1268658019904011E0FCA3FB
:10478600E0FDA3E0FEA3E02401FFE43EFEE43DFDE0
:10479600E43CFC90401112423D0245AE9040047448
:1047A60001F0904018E0F8A3E0F9A3E0FAA3E0FBDB
:1047B600E4FCFDEB2539FFEA3538FEED39FDEC3832
:1047C600FC90401812423DAF3DAE3CAD3BAC3A903A
:0747D60056CA12423D7F01AB
:0147DD0022B9
:0B665F00E0FCA3E0FDA3E0FEA3E0FFD1
:10666A008F328E318D308C2FE5207002FF229040C0
:10667A0004E07002FF22AF32AE31AD30AC2F904051
:10668A001812423D904009E0FCA3E0FDA3E0FEA3FE
:10669A00E0FF904018E0F8A3E0F9A3E0FAA3E0FBDA
:1066AA00D31241D140037F0022904018E0FCA3E0BE
:1066BA00FDA3E0FEA3E0FF125E78EF7006904004AF
:0666CA00F0FF227F012217
:0E08A4008F328E318D308C2F8B338A34893514
:1008B200E5207002FF22E532541FFFE4FEFDFCFB3F
:1008C200FAF9F8C31241D160037F0022E5322420F5
:1008D200FBE43531FAE43530F9E4352FF89056D699
:1008E200E0FEA3E0FFE4FCFDD31241D140037F0010
:1008F20022E4904004F0124F318E418F42C3E54210
:100902009402E541940050037F0022AB33AA34A93C
:100912003590001AE54212402BE54190001B12402F
:100922002B90001CE412402B90001DE412402B90EF
:10093200001EE412402B90001FE412402BE4907939
:1009420013F0900000E07002A3E06003020C21F5B6
:1009520039F53AD39056DBE0953A9056DAE095397C
:100962005003020C0CE4FCFD9056F2E0F8A3E0F90F
:10097200A3E0FAA3E0253AFFEA3539FEED39FDECB2
:1009820038FC755B01755C01755D57755E0B12680D
:10099200F5EF7002FF22E4F53FF540907915F0F58E
:1009A2003BF53CD39056D7E0953C9056D6E0953B2C
:1009B2005003020BAEE4FFFEFDFCAB32AA31A930BC
:1009C200A82F1241D16003020A4F740B253CF58215
:1009D2007457353BF583E0600764E56003020BA0C2
:1009E200E4F53DF53EAB33AA34A935853E82853D1B
:1009F20083123FECFFE53C253EFDE53B353DFC74B3
:100A02000B2DF58274573CF583EFF0053EE53E7001
:100A120002053D6420453D70CCE4FCFD9056F2E0B9
:100A2200F8A3E0F9A3E0FAA3E0253AFFEA3539FE9C
:100A3200ED39FDEC38FC755B01755C01755D577530
:100A42005E0B12692FEF7002FF22020B98E5404500
:100A52003F7006907914E53CF0740B253CF58274E6
:100A620057353BF583E0FFB4E50A0540E540702BBE
:100A7200053F8027EF701F0540E5407002053F7477
:100A82000B253CF5827457353BF58374E5F090797C
:100A9200157401F08005E4F53FF540E5322420FFAE
:100AA200E43531FEE43530FDE4352FFCC004C005E9
:100AB200C006C007E540AE3F7805C333CE33CED87B
:100AC200F9FBAA06E4F9F8D007D006D005D004C392
:100AD2001241D15003020BA0E4F53DF53EAE3DAF0D
:100AE2003EE4FCFDAB32AA31A930A82FD31241D18A
:100AF2004033AB36AA37A938853E82853D83123F03
:100B0200ECFF907914E07C00253EFDEC353DFC7451
:100B12000B2DF58274573CF583EFF0053EE53E70F0
:100B2200BC053D80B8E4F53DF53EAB33AA34A935AA
:100B3200853E82853D83123FECFF907914E0253299
:100B4200FDE43531CD253ECD353DFC740B2DF582CE
:100B520074573CF583EFF0053EE53E7002053D64B7
:100B620020453D70C5E4FCFD9056F2E0F8A3E0F9A3
:100B7200A3E0FAA3E0253AFFEA3539FEED39FDECB0
:100B820038FC755B01755C01755D57755E0B12690A
:100B92002FEF7002FF229079137401F0800E7420FF
:100BA200253CF53CE4353BF53B0209A5907913E081
:100BB20064016056E4FFFEFDFCAB32AA31A930A805
:100BC2002FC31241D16038907915E064017030FC76
:100BD200FD9056F2E0F8A3E0F9A3E0FAA3E0253A8B
:100BE200FFEA3539FEED39FDEC38FC755B01755CC9
:100BF20001755D57755E0B12692FEF7002FF2205BA
:100C02003AE53A70020539020955D39056DBE09570
:100C12003A9056DAE095394003020FF47F002290B1
:100C22000000E0FFA3E0904002CFF0A3EFF090407D
:100C320002E0FEA3E0FF1268659056A012423D90CA
:100C42004002E0F543A3E0F544E4F539F53A905665
:100C5200D8E0FFC3E53A9FE53994004003020F074D
:100C6200E4FCFD9056A0E0F8A3E0F9A3E0FAA3E0CB
:100C7200253AFFEA3539FEED39FDEC38FC755B01AA
:100C8200755C01755D57755E0B1268F5EF7002FFBA
:100C920022E4F53FF540907915F0F53BF53CD39011
:100CA20056D7E0953C9056D6E0953B5003020EA9EC
:100CB200E4FFFEFDFCAB32AA31A930A82F1241D1CC
:100CC2006003020D4A740B253CF5827457353BF5DF
:100CD20083E0600764E56003020E9BE4F53DF53EA8
:100CE200AB33AA34A935853E82853D83123FECFFA2
:100CF200E53C253EFDE53B353DFC740B2DF582744C
:100D0200573CF583EFF0053EE53E7002053D642059
:100D1200453D70CCE4FCFD9056A0E0F8A3E0F9A3B9
:100D2200E0FAA3E0253AFFEA3539FEED39FDEC3869
:100D3200FC755B01755C01755D57755E0B12692F61
:100D4200EF7002FF22020E93E540453F7006907954
:100D520014E53CF0740B253CF5827457353BF58362
:100D6200E0FFB4E50A0540E540702B053F8027EF20
:100D7200701F0540E5407002053F740B253CF5826B
:100D82007457353BF58374E5F09079157401F08062
:100D920005E4F53FF540E5322420FFE43531FEE479
:100DA2003530FDE4352FFCC004C005C006C007E5A0
:100DB20040AE3F7805C333CE33CED8F9FBAA06E462
:100DC200F9F8D007D006D005D004C31241D15003A0
:100DD200020E9BE4F53DF53EAE3DAF3EE4FCFDABBD
:100DE20032AA31A930A82FD31241D14033AB36AA4F
:100DF20037A938853E82853D83123FECFF907914F6
:100E0200E07C00253EFDEC353DFC740B2DF5827433
:100E1200573CF583EFF0053EE53E70BC053D80B8DA
:100E2200E4F53DF53EAB33AA34A935853E82853DD6
:100E320083123FECFF907914E02532FDE43531CD89
:100E4200253ECD353DFC740B2DF58274573CF58360
:100E5200EFF0053EE53E7002053D6420453D70C55C
:100E6200E4FCFD9056A0E0F8A3E0F9A3E0FAA3E0C9
:100E7200253AFFEA3539FEED39FDEC38FC755B01A8
:100E8200755C01755D57755E0B12692FEF7002FF7D
:100E9200229079137401F0800E7420253CF53CE415
:100EA200353BF53B020CA0907913E064016056E4F7
:100EB200FFFEFDFCAB32AA31A930A82FC31241D1EB
:100EC2006038907915E064017030FCFD9056A0E026
:100ED200F8A3E0F9A3E0FAA3E0253AFFEA3539FEE8
:100EE200ED39FDEC38FC755B01755C01755D57757C
:100EF2005E0B12692FEF7002FF22053AE53A70028B
:100F02000539020C50907913E064017003020FE27C
:100F1200904002E0FEA3E0FF1263C4904002EEF0B4
:100F2200A3EFF0D394EFEE94FF5003020FD0AF443F
:100F3200AE43126262904002EEF0A3EFF04E7002F6
:100F4200FF22904002E0FEA3E0FF1268659056A0E7
:100F520012423DE4F53BF53CD39056D7E0953C90E8
:100F620056D6E0953B4018740B253CF582745735F4
:100F72003BF583E4F0053CE53C70DD053B80D9E4BC
:100F8200F539F53A9056D8E0FFC3E53A9FE5399432
:100F920000503BE4FCFD9056A0E0F8A3E0F9A3E08A
:100FA200FAA3E0253AFFEA3539FEED39FDEC38FCCB
:100FB200755B01755C01755D57755E0B12692FEFEC
:100FC2007002FF22053AE53A70BA053980B6D3902D
:100FD2004003E094EF904002E094FF5003020C3093
:100FE200D3904003E094EF904002E094FF40037FEF
:100FF2000022AE41AF42E4FCFD90400512423D901A
:10100200400912424900000000904005E0FCA3E0C4
:10101200FDA3E0FEA3E0FF90400D12423D9040058B
:10102200A3A3E0FEA3E0FF12686590401112423DC7
:10103200E4904015F0A3F0A3F090400404F0904037
:10104200181242490000000090401C124249000060
:0410520000007F011A
:011056002277
:0E172C008F328E318D308C2F8B338A3489357D
:10173A00E5207002FF22904004E07002FF22E4904C
:10174A004004F0754001F541F53EF53FE4FFFEFD2A
:10175A00FCAB32AA31A930A82FD31241D1500302CF
:10176A001979904015E0FEA3E0FFEF2532FBEE3534
:10177A0031FAE43530F9E4352FF89056D6E0FEA375
:10178A00E0FFE4FCFDD31241D1400C9056D6E0F5BF
:10179A0036A3E0F5378010904016E02532F53790F1
:1017AA004015E03531F536D3904016E0940090406C
:1017BA0015E094005003021872904011E0FCA3E077
:1017CA00FDA3E0FEA3E0FF755B01755C01755D5743
:1017DA00755E0B1268F5EF700302186F904015E002
:1017EA00FEA3E0FFC3E5379FF537E5369EF536E4FD
:1017FA00F53AF53BC3E53B9537E53A95365034ABB8
:10180A0033AA34A935853B82853A83123FECFF908F
:10181A004016E0253BFD904015E0353AFC740B2D4F
:10182A00F58274573CF583EFF0053BE53B70C5053F
:10183A003A80C1904011E0FCA3E0FDA3E0FEA3E0E2
:10184A00FF755B01755C01755D57755E0B12692F3B
:10185A00EF7002FF22904016E02537F0904015E025
:10186A003536F080367F0022904011E0FCA3E0FD7F
:10187A00A3E0FEA3E0FF755B01E535253FF9E534FA
:10188A00353E85335CF55D895E12692FEF7002FF84
:10189A0022904015E536F0A3E537F0AE36AF37AB08
:1018AA0007AA06C3E5329BF532E5319AF531E530F0
:1018BA009400F530E52F9400F52FE537253FF53FE5
:1018CA00E536353EF53E9056D7E024FFFF9056D6D2
:1018DA00E034FFFE904015E0FCA3E0FDD39FEC9EB0
:1018EA0050030217569056D6E0FEA3E0FFED9FFF85
:1018FA00EC9E904015F0A3EFF0A3E004F09056D8C8
:10190A00E014FF904017E0D39F4042E4F090400D6E
:10191A00A3A3E0FEA3E0FF126262E4FCFD90400D87
:10192A0012423DE4FFFEFDFC90400DE0F8A3E0F911
:10193A00A3E0FAA3E0FBC31241D17002FF22904058
:10194A000DA3A3E0FEA3E0FF126865801990401181
:10195A00E0FCA3E0FDA3E0FEA3E02401FFE43EFED9
:10196A00E43DFDE43CFC90401112423D02175690C2
:10197A004018E0F8A3E0F9A3E0FAA3E0FBE4FCFDD9
:10198A00EB253FFFEA353EFEED39FDEC38FC904091
:10199A001812423D7FC8126A68E54064016003027A
:1019AA001D81900000E07002A3E06003021B73F542
:1019BA0038F539D39056DBE095399056DAE0953808
:1019CA005003021D81E4FCFD9056F2E0F8A3E0F911
:1019DA00A3E0FAA3E02539FFEA3538FEED39FDEC3C
:1019EA0038FC755B01755C01755D57755E0B126895
:1019FA00F5EF7002FF22E4F53AF53BD39056D7E0B3
:101A0A00953B9056D6E0953A5003021B5F74252504
:101A1A003BF5827457353AF583E0FF7E007426253C
:101A2A003BF5827457353AF583E0FD7C00126A383B
:101A3A008E3C8F3DE4FCFD904005E0F8A3E0F9A35D
:101A4A00E0FAA3E0FBC31241D16003021B51740BFD
:101A5A00253BF5827457353AF583E064E570030255
:101A6A001B51904009E0FCA3E0FDA3E0FEA3E0FFC8
:101A7A00904018E0F8A3E0F9A3E0FAA3E0FBD31240
:101A8A0041D14014904018E0FCA3E0FDA3E0FEA37E
:101A9A00E0FF90400912423D904009A3A3A3E0FF52
:101AAA007427253BF5827457353AF583EFF0904059
:101ABA0009E0FCA3E0FDA3E0FEA3E0FF78081241E1
:101ACA00E27428253BF5827457353AF583EFF09096
:101ADA004009E0FCA3E0FDA3E0FEA3E0FF781012BA
:101AEA0041E27429253BF5827457353AF583EFF0C4
:101AFA00904009E0FCA3E0FDA3E0FEA3E0FF781814
:101B0A001241E2742A253BF5827457353AF583EF80
:101B1A00F0E4FCFD9056F2E0F8A3E0F9A3E0FAA3A2
:101B2A00E02539FFEA3538FEED39FDEC38FC755B06
:101B3A0001755C01755D57755E0B12692FEF7002B6
:101B4A00FF22754101800E7420253BF53BE4353AAE
:101B5A00F53A021A05E54164017003021D8105394F
:101B6A00E539700205380219BD900000E0FFA3E0D4
:101B7A00904002CFF0A3EFF0904002E0FEA3E0FF16
:101B8A001268659056A012423DE4F538F539905630
:101B9A00D8E0FFC3E5399FE53894004003021D4BA6
:101BAA00E4FCFD9056A0E0F8A3E0F9A3E0FAA3E074
:101BBA002539FFEA3538FEED39FDEC38FC755B0155
:101BCA00755C01755D57755E0B1268F5EF7002FF63
:101BDA0022E4F53AF53BD39056D7E0953B9056D69A
:101BEA00E0953A5003021D3A7425253BF582745755
:101BFA00353AF583E0FF7E007426253BF58274575B
:101C0A00353AF583E0FD7C00126A388E3C8F3DE45C
:101C1A00FCFD904005E0F8A3E0F9A3E0FAA3E0FB9D
:101C2A00C31241D16003021D2C740B253BF582744B
:101C3A0057353AF583E064E57003021D2C9040099C
:101C4A00E0FCA3E0FDA3E0FEA3E0FF904018E0F86B
:101C5A00A3E0F9A3E0FAA3E0FBD31241D140149028
:101C6A004018E0FCA3E0FDA3E0FEA3E0FF904009DA
:101C7A0012423D904009A3A3A3E0FF7427253BF538
:101C8A00827457353AF583EFF0904009E0FCA3E0FF
:101C9A00FDA3E0FEA3E0FF78081241E27428253B89
:101CAA00F5827457353AF583EFF0904009E0FCA3CA
:101CBA00E0FDA3E0FEA3E0FF78101241E2742925BB
:101CCA003BF5827457353AF583EFF0904009E0FC12
:101CDA00A3E0FDA3E0FEA3E0FF78181241E2742A14
:101CEA00253BF5827457353AF583EFF0E4FCFD9015
:101CFA0056A0E0F8A3E0F9A3E0FAA3E02539FFEA49
:101D0A003538FEED39FDEC38FC755B01755C017503
:101D1A005D57755E0B12692FEF7002FF2275410144
:101D2A00800E7420253BF53BE4353AF53A021BE078
:101D3A00E5416401600B0539E53970020538021B7B
:101D4A0098E5416401601E904002E0FEA3E0FF12A4
:101D5A0063C4904002EEF0A3EFF0D394EFEE94FF49
:101D6A005003021B82D3904003E094EF904002E0BC
:0E1D7A0094FF40037F00229040047401F0FFAC
:011D88002238
:06328E008B2F8A3089310C
:10329400E5207002FF22900000E07002A3E06003CA
:1032A40002345BF532F533D39056DBE09533905618
:1032B400DAE095325003023446E4FCFD9056F2E025
:1032C400F8A3E0F9A3E0FAA3E02533FFEA3532FEE0
:1032D400ED39FDEC38FC755B01755C01755D577566
:1032E4005E0B1268F5EF7002FF22E4F534F535D376
:1032F4009056D7E095359056D6E095345003023475
:1033040032740B2535F58274573534F583E0700239
:10331400FF22E4F537AB2FAA30A9318537827583B4
:1033240000123FECFFE5377C002535FDEC3534FC1D
:10333400740B2DF58274573CF583E0B50709053706
:10334400E537D3940A40CEE537D3940A50030234C8
:1033540024740B2535F58274573534F58374E5F000
:1033640074252535F58274573534F583E0FF7E00E6
:1033740074262535F58274573534F583E0FD7C00D9
:10338400126A38E4FCFD90400512423DE53524E024
:10339400F539E53434FFF538C3E53864809480406A
:1033A4002D74162539F58274573538F583E0B40F3A
:1033B4001D740B2539F58274573538F58374E5F09F
:1033C40074E02539F53974FF3538F53880CA7F0F34
:1033D400126A68E4FCFD9056F2E0F8A3E0F9A3E079
:1033E400FAA3E02533FFEA3532FEED39FDEC38FC73
:1033F400755B01755C01755D57755E0B12692FEF86
:103404007002FF227F0A126A68904005A3A3E0FEBF
:10341400A3E0FF125F8CEF7002FF22753601800E6D
:1034240074202535F535E43534F5340232F3E536C8
:103434006401600E0533E53360030232AB053202EA
:1034440032ABD39056DBE095339056DAE0953240B8
:103454000302364E7F0022900000E0FFA3E090407C
:1034640002CFF0A3EFF0904002E0FEA3E0FF126869
:10347400659056A012423DE4F532F5339056D8E0FB
:10348400FFC3E5339FE53294004003023618E4FCA1
:10349400FD9056A0E0F8A3E0F9A3E0FAA3E02533F9
:1034A400FFEA3532FEED39FDEC38FC755B01755CE5
:1034B40001755D57755E0B1268F5EF7002FF22E42B
:1034C400F534F535D39056D7E095359056D6E0953A
:1034D400345003023607740B2535F582745735349E
:1034E400F583E07002FF22E4F537AB2FAA30A9314F
:1034F400853782758300123FECFFE5377C00253564
:10350400FDEC3534FC740B2DF58274573CF583E0E7
:10351400B507090537E537D3940A40CEE537D39488
:103524000A50030235F9740B2535F5827457353486
:10353400F58374E5F074252535F58274573534F533
:1035440083E0FF7E0074262535F58274573534F503
:1035540083E0FD7C00126A38E4FCFD9040051242D1
:103564003DE53524E0F539E53434FFF538C3E53875
:1035740064809480402D74162539F582745735384B
:10358400F583E0B40F1D740B2539F5827457353873
:10359400F58374E5F074E02539F53974FF3538F5B1
:1035A4003880CA7F0F126A68E4FCFD9056A0E0F8E8
:1035B400A3E0F9A3E0FAA3E02533FFEA3532FEEDF8
:1035C40039FDEC38FC755B01755C01755D57755E02
:1035D4000B12692FEF7002FF227F0A126A68904073
:1035E40005A3A3E0FEA3E0FF125F8CEF7002FF22AD
:1035F400753601800E74202535F535E43534F534FF
:103604000234C8E5366401600B0533E53370020506
:1036140032023480E5366401601E904002E0FEA36D
:10362400E0FF1263C4904002EEF0A3EFF0D394EFF6
:10363400EE94FF500302346AD3904003E094EF9079
:0C3644004002E094FF40037F00227F0161
:013650002257
:1058D100E5207002FF229056EEA3A3E0FEA3E08E26
:1058E1002FF530E4F538F537F536F5359056E0E02B
:1058F100FEA3E0FFE4FCFD9056EEE0F8A3E0F9A37F
:10590100E0FAA3E02FFBEA3EFAED39F9EC38F8AE04
:105911002FAF30E4D31241D14072AE2FAF30E4FC4F
:10592100FD755B01755C01755D57755E0B1268F560
:10593100EF6048E4FBFAD39056D7E09B9056D6E04F
:105941009A403B740B2BF58274573AF583E0702231
:10595100740C2BF58274573AF583E07015E5382401
:1059610001F538E43537F537E43536F536E43535C4
:10597100F53574022BFBE43AFA80BB7F0022053037
:10598100E53060030258ED052F0258ED9056D8E03E
:10599100FF7E009056D6E0FCA3E0FD12404DE48F5F
:1059A100348E33F532F531AD32AC31AB38AA37A98B
:1059B10036A8351240B48F348E338D328C3178183D
:1059C1001241E2900002EFF0AF34AE33AD32AC31B0
:1059D10078101241E2A3EFF0AF34AE33AD32AC3107
:1059E10078081241E2A3EFF0E534FFA3EFF09056FF
:0A59F100CA124249000000047F01C1
:0159FB002289
:0E0026008F328E318D308C2F8B338A3489359A
:10003400E5207002FF22E532541FFFE4FEFDFCFBC5
:10004400FAF9F8C31241D160037F0022E53224207B
:10005400FBE43531FAE43530F9E4352FF89056D61F
:10006400E0FEA3E0FFE4FCFDD31241D140037F0096
:1000740022E4904004F090401C1242490000000029
:10008400124F318E418F42C3E5429402E541940000
:1000940050037F0022AB33AA34A93590000B7410AF
:1000A40012402B90001AE54212402BE54190001BB0
:1000B40012402B90001CE412402B90001DE41240CF
:1000C4002B90001EE412402B90001FE412402BE4FE
:1000D400907913F0900000E07002A3E06003020343
:1000E400B5F539F53AD39056DBE0953A9056DAE017
:1000F400953950030203A0E4FCFD9056F2E0F8A306
:10010400E0F9A3E0FAA3E0253AFFEA3539FEED3938
:10011400FDEC38FC755B01755C01755D57755E0B14
:100124001268F5EF7002FF22E4F53FF5409079156F
:10013400F0F53BF53CD39056D7E0953C9056D6E08D
:10014400953B5003020342E4FFFEFDFCAB32AA31AF
:10015400A930A82F1241D160030201E3740B253C9E
:10016400F5827457353BF583E0600764E56003026C
:100174000334E4F53DF53EAB33AA34A935853E821C
:10018400853D83123FECFFE53C253EFDE53B353DD7
:10019400FC740B2DF58274573CF583EFF0053EE5B6
:1001A4003E7002053D6420453D70CCE4FCFD905654
:1001B400F2E0F8A3E0F9A3E0FAA3E0253AFFEA3578
:1001C40039FEED39FDEC38FC755B01755C01755D3C
:1001D40057755E0B12692FEF7002FF2202032CE5A4
:1001E40040453F7006907914E53CF0740B253CF5CE
:1001F400827457353BF583E0FFB4E50A0540E540DA
:10020400702B053F8027EF701F0540E54070020505
:100214003F740B253CF5827457353BF58374E5F048
:100224009079157401F08005E4F53FF540E532243A
:1002340020FFE43531FEE43530FDE4352FFCC00405
:10024400C005C006C007E540AE3F7805C333CE33D2
:10025400CED8F9FBAA06E4F9F8D007D006D005D029
:1002640004C31241D15003020334E4F53DF53EAE1C
:100274003DAF3EE4FCFDAB32AA31A930A82FD31226
:1002840041D14033AB36AA37A938853E82853D83B8
:10029400123FECFF907914E07C00253EFDEC353DE7
:1002A400FC740B2DF58274573CF583EFF0053EE5A5
:1002B4003E70BC053D80B8E4F53DF53EAB33AA3451
:1002C400A935853E82853D83123FECFF907914E089
:1002D4002532FDE43531CD253ECD353DFC740B2D65
:1002E400F58274573CF583EFF0053EE53E70020558
:1002F4003D6420453D70C5E4FCFD9056F2E0F8A352
:10030400E0F9A3E0FAA3E0253AFFEA3539FEED3936
:10031400FDEC38FC755B01755C01755D57755E0B12
:1003240012692FEF7002FF229079137401F0800E8E
:100334007420253CF53CE4353BF53B0201399079CA
:1003440013E064016056E4FFFEFDFCAB32AA31A960
:1003540030A82FC31241D16038907915E064017040
:1003640030FCFD9056F2E0F8A3E0F9A3E0FAA3E034
:10037400253AFFEA3539FEED39FDEC38FC755B01B1
:10038400755C01755D57755E0B12692FEF7002FF86
:1003940022053AE53A700205390200E9D39056DBAA
:1003A400E0953A9056DAE0953940030207887F00D9
:1003B40022900000E0FFA3E0904002CFF0A3EFF012
:1003C400904002E0FEA3E0FF1268659056A012423E
:1003D4003D904002E0F543A3E0F544E4F539F53AF5
:1003E4009056D8E0FFC3E53A9FE5399400400302F4
:1003F400069BE4FCFD9056A0E0F8A3E0F9A3E0FA24
:10040400A3E0253AFFEA3539FEED39FDEC38FC75F9
:100414005B01755C01755D57755E0B1268F5EF70D5
:1004240002FF22E4F53FF540907915F0F53BF53CE9
:10043400D39056D7E0953C9056D6E0953B500302B6
:10044400063DE4FFFEFDFCAB32AA31A930A82F1211
:1004540041D160030204DE740B253CF582745735E8
:100464003BF583E0600764E5600302062FE4F53D95
:10047400F53EAB33AA34A935853E82853D83123FD0
:10048400ECFFE53C253EFDE53B353DFC740B2DF5CD
:100494008274573CF583EFF0053EE53E7002053D5E
:1004A4006420453D70CCE4FCFD9056A0E0F8A3E048
:1004B400F9A3E0FAA3E0253AFFEA3539FEED39FD68
:1004C400EC38FC755B01755C01755D57755E0B124C
:1004D400692FEF7002FF22020627E540453F7006B0
:1004E400907914E53CF0740B253CF5827457353B48
:1004F400F583E0FFB4E50A0540E540702B053F8035
:1005040027EF701F0540E5407002053F740B253C42
:10051400F5827457353BF58374E5F09079157401D1
:10052400F08005E4F53FF540E5322420FFE4353161
:10053400FEE43530FDE4352FFCC004C005C006C020
:1005440007E540AE3F7805C333CE33CED8F9FBAAD6
:1005540006E4F9F8D007D006D005D004C31241D17F
:10056400500302062FE4F53DF53EAE3DAF3EE4FCFC
:10057400FDAB32AA31A930A82FD31241D14033ABFD
:1005840036AA37A938853E82853D83123FECFF9019
:100594007914E07C00253EFDEC353DFC740B2DF513
:1005A4008274573CF583EFF0053EE53E70BC053D93
:1005B40080B8E4F53DF53EAB33AA34A935853E82D7
:1005C400853D83123FECFF907914E02532FDE4353C
:1005D40031CD253ECD353DFC740B2DF58274573C51
:1005E400F583EFF0053EE53E7002053D6420453D90
:1005F40070C5E4FCFD9056A0E0F8A3E0F9A3E0FA8E
:10060400A3E0253AFFEA3539FEED39FDEC38FC75F7
:100614005B01755C01755D57755E0B12692FEF7098
:1006240002FF229079137401F0800E7420253CF5AA
:100634003CE4353BF53B020434907913E0640160FB
:1006440056E4FFFEFDFCAB32AA31A930A82FC31239
:1006540041D16038907915E064017030FCFD90560A
:10066400A0E0F8A3E0F9A3E0FAA3E0253AFFEA3515
:1006740039FEED39FDEC38FC755B01755C01755D87
:1006840057755E0B12692FEF7002FF22053AE53AA7
:10069400700205390203E4907913E06401700302E7
:1006A4000776904002E0FEA3E0FF1263C49040028C
:1006B400EEF0A3EFF0D394EFEE94FF50030207643F
:1006C400AF44AE43126262904002EEF0A3EFF04EEC
:1006D4007002FF22904002E0FEA3E0FF12686590E2
:1006E40056A012423DE4F53BF53CD39056D7E09535
:1006F4003C9056D6E0953B4018740B253CF582742B
:1007040057353BF583E4F0053CE53C70DD053B8063
:10071400D9E4F539F53A9056D8E0FFC3E53A9FE5B8
:10072400399400503BE4FCFD9056A0E0F8A3E0F9B6
:10073400A3E0FAA3E0253AFFEA3539FEED39FDECF2
:1007440038FC755B01755C01755D57755E0B12694C
:100754002FEF7002FF22053AE53A70BA053980B6E8
:10076400D3904003E094EF904002E094FF500302E2
:1007740003C4D3904003E094EF904002E094FF4020
:10078400037F0022753B00753C40D39056D7E0951B
:100794003C9056D6E0953B4018740B253CF582748A
:1007A40057353BF583E4F0053CE53C70DD053B80C3
:1007B400D9E4F53BF53C740B253CF5827457353B85
:1007C400F5837420F0053CE53C7002053B642B4541
:1007D4003B70E390570B742EF0753B00753C0BABEC
:1007E40033AA34A935853C82853B83123FECFF74E0
:1007F4000B253CF5827457353BF583EFF0053CE55A
:100804003C7002053B6420453B70D490572B742EFA
:10081400F0A3F0753B00753C2BAB33AA34A935E546
:100824003C24E0FFE53B34FF8F82F583123FECFF6D
:10083400740B253CF5827457353BF583EFF0053C8A
:10084400E53C7002053B6440453B70CD900000E000
:10085400FEA3E0905745F0EEA3F0AF42AE4112681C
:10086400659056A012423D9056A0E0FCA3E0FDA383
:10087400E0FEA3E0FF755B01755C01755D57755E75
:100884000B12692FEF7002FF22900000E541F0A3E4
:0F089400E542F090400D124249000000007F0144
:0108A3002232
:064CC5007B017A5679A97B
:064CCB008B2F8A308931B5
:104CD100E5207002FF22E4904004F0F535900000D9
:104CE100E07002A3E06003024DD3F536D39056DBAA
:104CF100E095369056DAE094005003024DBEE4FC94
:104D0100FDFE9056F2E0F8A3E0F9A3E0FAA3E02556
:104D110036FFEE3AFEED39FDEC38FC755B01755C52
:104D210001755D57755E0B1268F5EF7002FF22E4A5
:104D3100F532F533D39056D7E095339056D6E095BA
:104D410032406F740B2533F58274573532F583E0A9
:104D51007002FF22E4F534AB2FAA30A931853482E9
:104D6100758300123FECFFE5347C002533FDEC3503
:104D710032FC740B2DF58274573CF583E0B50709BD
:104D81000534E534D3940A40CEE534D3940A401572
:104D910074162533F58274573532F583E030E40516
:104DA100753501800D74202533F533E43532F53244
:104DB1008082E535640160050536024CEDD39056DD
:104DC100DBE095369056DAE0940050037F00220232
:104DD1004EF9900000E0FFA3E0904002CFF0A3EF76
:104DE100F0904002E0FEA3E0FF1268659056A01229
:104DF100423DE4F5369056D8E0FFE536C39F4003C7
:104E0100024EC3E4FCFDFE9056A0E0F8A3E0F9A336
:104E1100E0FAA3E02536FFEE3AFEED39FDEC38FC71
:104E2100755B01755C01755D57755E0B1268F5EF79
:104E31007002FF22E4F532F533D39056D7E0953373
:104E41009056D6E09532406F740B2533F582745736
:104E51003532F583E07002FF22E4F534AB2FAA303E
:104E6100A931853482758300123FECFFE5347C0063
:104E71002533FDEC3532FC740B2DF58274573CF56E
:104E810083E0B507090534E534D3940A40CEE5340F
:104E9100D3940A401574162533F58274573532F5CB
:104EA10083E030E405753501800D74202533F53339
:104EB100E43532F5328082E535640160050536025C
:104EC1004DF6E5356401601E904002E0FEA3E0FF6F
:104ED1001263C4904002EEF0A3EFF0D394EFEE948E
:104EE100FF5003024DE2D3904003E094EF90400263
:104EF100E094FF40037F002274252533F582745727
:104F01003532F583E0FF7E0074262533F582745730
:104F11003532F583E0FD7C00126A38900000EEF036
:0F4F2100A3EFF090400D124249000000007F0105
:014F3000225E
:1065E200E5207002FF22900000E0FCA3E0FD4C7069
:1065F200037F0122E4904004F0AF05AE0412686507
:106602009056A012423D9056A0E0FCA3E0FDA3E00C
:10661200FEA3E0FF755B01755C01755D57755E0B4E
:106622001268F5EF7002FF2290572BE0642E60098A
:10663200A3E0642E60037F0022905745E0FF7E00B6
:10664200A3E0FD7C00126A38900000EEF0A3EFF0A8
:0D66520090400D124249000000007F01221F
:106A2400E5207002FF22E4904004F0900000F0A3FF
:046A3400F07F0122CC
:105B2300E49056C9F0A3124249000000009056A425
:105B3300E0B40D004003025C44905B43F8282873F3
:105B4300025B6A025B6F025B74025B8E025B97020D
:105B53005BCC025BE5025BF5025BFA025C06025C6E
:105B630032025C37025C3C123CC7805A1247DE802B
:105B7300559056A5E0FCA3E0FDA3E0FEA3E0FF7B68
:105B8300017A007902124286025C3F9056A51266A2
:105B9300D0025C3F1247DE9056C9EFF06008904098
:105BA300091266D080209056A5E0FCA3E0FDA3E097
:105BB300FEA3E0FF7536017537007538027B017A65
:105BC3005679A9121D89025C3F9056A5E0FCA3E01B
:105BD300FDA3E0FEA3E0FF7B017A007902122D7A98
:105BE300805AE4904004F07B017A5679A9124A580E
:105BF300804A1257768045E52060469056C9740165
:105C0300F0803E12511D9056C9EFF070349056A5A6
:105C1300E0FCA3E0FDA3E0FEA3E0FF7536017537CA
:105C2300007538027B017A5679A9121057800D123C
:105C3300511D800812609A800312698C9056C9EF37
:075C4300F01264517F012201
:103CC700E5207002FF22E4F52FF530F533F535F5E1
:103CD70031F53290402075F020E53212427AE53115
:103CE70075F020A425832532F583E4F090402175F3
:103CF700F020E53212427AE53175F020A42583F8E9
:103D07002532F583E4F00532E5327002053164149B
:103D1700453170BF907930E0FCA3E0FDA3E0FEA33E
:103D2700E0FFA312423D907934E0FCA3E0FDA3E05D
:103D3700FEA3E0FF1267A89056A012423DE4F534B7
:103D47009056D8E0FFE534C39F4003023F77E4FC79
:103D5700FDFE9056A0E0F8A3E0F9A3E0FAA3E02562
:103D670034FFEE3AFEED39FDEC38FC755B01755C0E
:103D770001755D57755E0B1268F5EF7002FF22E45F
:103D8700F531F532D39056D7E095329056D6E09577
:103D9700315003023F6C740B2532F582745735316D
:103DA700F583E0FF70028052EF64E57003023F5E27
:103DB700E4F9E9FD7C002532FFEC3531FE740B2F69
:103DC700F58274573EF583E0FBE530AE2F7805C3E7
:103DD70033CE33CED8F92DFFEE3CFE74022FF58299
:103DE70074003EF583EBF009B920C70530E5307064
:103DF70002052FC3E52F94024006753301023F6C7D
:103E0700E535C394144003023F5E74162532F582EC
:103E170074573531F583E0640F6003023F20740B5C
:103E27002532F58274573531F583E0541F1475F048
:103E37001AA4F537D394E04003023F5EE4F53679E0
:103E470001E97E002532FFEE3531FE740B2FF58236
:103E570074573EF583E0FFE536FDE5372DFDE43386
:103E6700FC75F020E535A42420F582E5F03440F513
:103E7700832535F583E5822DF582E5833CF583EFD0
:103E8700F0053609B90BBA790EE97E002532FFEE47
:103E97003531FE740B2FF58274573EF583E0FFE54D
:103EA70036FDE5372DFDE433FC75F020E535A42418
:103EB70020F582E5F03440F5832535F583E5822D3D
:103EC700F582E5833CF583EFF0053609B91ABA792F
:103ED7001CE97E002532FFEE3531FE740B2FF5828B
:103EE70074573EF583E0FFE536FDE5372DFDE433F6
:103EF700FC75F020E535A42420F582E5F03440F583
:103F0700832535F583E5822DF582E5833CF583EF3F
:103F1700F0053609B920BA803EE4F9E97E0025327A
:103F2700FFEE3531FE740B2FF58274573EF583E0B3
:103F3700FF75F020E535A42420F582E5F03441F53E
:103F4700832535F583E58229F582E43583F583EF0B
:103F5700F009B920C6053574202532F532E435312C
:103F6700F531023D8BE533640160050534023D47B9
:103F7700E5336401603C907934E0FCA3E0FDA3E005
:103F8700FEA3E0FF12618A90793412423D905702F6
:103F9700E0FCA3E0FDA3E0FEA3E0FF907934E0F8A6
:103FA700A3E0F9A3E0FAA3E0FBD31241D150030247
:103FB7003D2DE530AE2F7805C333CE33CED8F9FF8C
:0B3FC700E4FCFD9056CA12423D7F0151
:013FD20022CC
:0647DE007B017A5679A967
:0647E4008B2F8A308931A1
:1047EA00E5207002FF22E4904004F0907930E0FC6A
:1047FA00A3E0FDA3E0FEA3E0FFA312423D907934BB
:10480A00E0FCA3E0FDA3E0FEA3E0FF1267A8905638
:10481A00A012423DE4F5369056D8E0FFE536C39F34
:10482A004003024920E4FCFDFE9056A0E0F8A3E014
:10483A00F9A3E0FAA3E02536FFEE3AFEED39FDECE6
:10484A0038FC755B01755C01755D57755E0B126806
:10485A00F5EF7002FF22E4F532F533D39056D7E034
:10486A0095339056D6E095325003024915740B25BC
:10487A0033F58274573532F583E07002FF22E4F58E
:10488A0034AB2FAA30A931853482758300123FECEC
:10489A00FFE5347C002533FDEC3532FC740B2DF535
:1048AA008274573CF583E0B507090534E534D3949F
:1048BA000A40CEE534D3940A404374162533F58270
:1048CA0074573532F583E020E433E4F5347E00E5AD
:1048DA00332534FFEE3532FE740B2FF58274573EC2
:1048EA00F583E0FF74022534F582E43400F583EFA2
:1048FA00F00534E534B420D5753501800E742025D1
:10490A0033F533E43532F532024865E53564016042
:10491A00050536024821E5356401603C907934E0AA
:10492A00FCA3E0FDA3E0FEA3E0FF12618A907934C4
:10493A0012423D905702E0FCA3E0FDA3E0FEA3E093
:10494A00FF907934E0F8A3E0F9A3E0FAA3E0FBD3FF
:10495A001241D15003024807905702E0FCA3E0FD40
:10496A00A3E0FEA3E0FF907934E0F8A3E0F9A3E026
:10497A00FAA3E0FBD31241D140037F002290400406
:10498A007401F090001CE0FFE4FCFDFEC007A3E008
:10499A00FFE48F5CF55BF55AF559900016E0FFE4E9
:1049AA008F60F55FF55EF55DA3E0FFE48F64F56364
:1049BA00F562F561D00712656190400512423D909B
:1049CA00001EE0FFE4FCFDFEC007A3E0FFE48F5CED
:1049DA00F55BF55AF559A3E0FFE48F60F55FF55EE4
:1049EA00F55DA3E0FFE48F64F563F562F561D00736
:1049FA0012656190400912423D904005E0FCA3E037
:104A0A00FDA3E0FEA3E0FF90400D12423D90400559
:104A1A00E0FCA3E0FDA3E0FEA3E0FF1267A890403C
:104A2A001112423DE4904015F0A3F0A3F090401C0F
:104A3A00124249000000009040181242490000004A
:0D4A4A00009056CA124249000000207F0172
:014A5700223C
:0E4286008F328E318D308C2F8B338A348935F8
:10429400E5207002FF22904004E07002FF22853284
:1042A4003D85313C85303B852F3AE4F538F539FFBF
:1042B4007E40FDFCAB32AA31A930A82FD31241D1E4
:1042C40040037F0022904018E0FCA3E0FDA3E0FE41
:1042D400A3E02532FFEE3531FEED3530FDEC352F10
:1042E400FC904009E0F8A3E0F9A3E0FAA3E0FBC3E3
:1042F4001241D150037F0022E4FFFEFDFCAB32AA41
:1043040031A930A82FD31241D150030244FC90406C
:1043140015E0FEA3E0FFEF2532FBEE3531FAE4357C
:1043240030F9E4352FF89056D6E0FEA3E0FFE4FC24
:10433400FDD31241D1400C9056D6E0F536A3E0F5FA
:10434400378010904016E02532F537904015E0355F
:1043540031F536D3904016E09400904015E0940077
:1043640050030243E6904011E0FCA3E0FDA3E0FE0D
:10437400A3E0FF755B01755C01755D57755E0B12FB
:1043840068F5EF605A904015E0FEA3E0FFC3E537FF
:104394009FF537E5369EF536E4FFFEC3EF9537EE1D
:1043A4009536502B904016E02FFD904015E03EFCD2
:1043B400740B2DF58274573CF583E0AB33AA34A912
:1043C400358F828E8312402B0FBF00010E80CC905C
:1043D4004016E02537F0904015E03536F080367F02
:1043E4000022904011E0FCA3E0FDA3E0FEA3E0FF67
:1043F400755B01E5352539F9E534353885335CF5E8
:104404005D895E1268F5EF7002FF22904015E53673
:10441400F0A3E537F0AE36AF37AB07AA06C3E532F3
:104424009BF532E5319AF531E5309400F530E52F0E
:104434009400F52FE5372539F539E5363538F53863
:104444009056D7E024FFFF9056D6E034FFFE90400C
:1044540015E0FCA3E0FDD39FEC9E50030242FC90C8
:1044640056D6E0FEA3E0FFED9FFFEC9E904015F0D2
:10447400A3EFF0A3E004F09056D8E014FF904017A7
:10448400E0D39F4051E4F090400DE0FCA3E0FDA395
:10449400E0FEA3E0FF12618A90400D12423D905766
:1044A40002E0FCA3E0FDA3E0FEA3E0FF90400DE0EA
:1044B400F8A3E0F9A3E0FAA3E0FBD31241D140034F
:1044C4007F002290400DE0FCA3E0FDA3E0FEA3E00A
:1044D400FF1267A88019904011E0FCA3E0FDA3E05F
:1044E400FEA3E02401FFE43EFEE43DFDE43CFC9039
:1044F400401112423D0242FC9040047401F090408D
:1045040018E0F8A3E0F9A3E0FAA3E0FBE4FCFDEB78
:104514002539FFEA3538FEED39FDEC38FC904018BA
:1045240012423DAF3DAE3CAD3BAC3A9056CA12424E
:034534003D7F01C7
:014537002261
:0B66D000E0FCA3E0FDA3E0FEA3E0FF60
:1066DB008F328E318D308C2FE5207002FF2290404F
:1066EB0004E07002FF22AF32AE31AD30AC2F9040E0
:1066FB001812423D904009E0FCA3E0FDA3E0FEA38D
:10670B00E0FF904018E0F8A3E0F9A3E0FAA3E0FB68
:10671B00D31241D140037F0022904018E0FCA3E04C
:10672B00FDA3E0FEA3E0FF125C4AEF70069040046D
:06673B00F0FF227F0122A5
:0E1D89008F328E318D308C2F8B338A3489351A
:101D9700E5207002FF22E532541FFFE4FEFDFCFB45
:101DA700FAF9F8C31241D160037F0022E5322420FB
:101DB700FBE43531FAE43530F9E4352FF89056D69F
:101DC700E0FEA3E0FFE4FCFDD31241D140037F0016
:101DD70022E4904004F01239908F448E438D428C58
:101DE70041E47F02FEFDFCAB44AA43A942A841C3DC
:101DF7001241D150037F0022AF44AE43AD42AC4104
:101E070078181241E2AB33AA34A935900015EF12C6
:101E1700402BAF44AE43AD42AC4178101241E29043
:101E27000014EF12402BAF44AE43AD42AC417808EB
:101E37001241E290001BEF12402B90001AE544126A
:101E4700402B90001CE412402B90001DE412402B05
:101E570090001EE412402B90001FE412402BE490E8
:101E67007913F0907930E0FCA3E0FDA3E0FEA3E056
:101E7700FFA312423D907934E0FCA3E0FDA3E0FE0E
:101E8700A3E0FF1267A89056A012423D907934E074
:101E9700FCA3E0FDA3E0FEA3E0F5488E478D468C4A
:101EA70045E4F539F53A9056D8E0FFC3E53A9FE5A2
:101EB7003994004003022164E4FCFD9056A0E0F849
:101EC700A3E0F9A3E0FAA3E0253AFFEA3539FEEDEE
:101ED70039FDEC38FC755B01755C01755D57755E06
:101EE7000B1268F5EF7002FF22E4F53FF540907999
:101EF70015F0F53BF53CD39056D7E0953C9056D678
:101F0700E0953B5003022106E4FFFEFDFCAB32AA3D
:101F170031A930A82F1241D16003021FA7740B25E6
:101F27003CF5827457353BF583E0600764E5600351
:101F37000220F8E4F53DF53EAB33AA34A935853EDA
:101F470082853D83123FECFFE53C253EFDE53B35B1
:101F57003DFC740B2DF58274573CF583EFF0053E7D
:101F6700E53E7002053D6420453D70CCE4FCFD90E4
:101F770056A0E0F8A3E0F9A3E0FAA3E0253AFFEAC8
:101F87003539FEED39FDEC38FC755B01755C017583
:101F97005D57755E0B12692FEF7002FF220220F06A
:101FA700E540453F7006907914E53CF0740B253CFD
:101FB700F5827457353BF583E0FFB4E50A0540E544
:101FC70040702B053F8027EF701F0540E5407002EA
:101FD700053F740B253CF5827457353BF58374E553
:101FE700F09079157401F08005E4F53FF540E5328E
:101FF7002420FFE43531FEE43530FDE4352FFCC005
:1020070004C005C006C007E540AE3F7805C333CE20
:1020170033CED8F9FBAA06E4F9F8D007D006D005E5
:10202700D004C31241D150030220F8E4F53DF53E38
:10203700AE3DAF3EE4FCFDAB32AA31A930A82FD3A9
:102047001241D14033AB36AA37A938853E82853D48
:1020570083123FECFF907914E07C00253EFDEC35C0
:102067003DFC740B2DF58274573CF583EFF0053E6C
:10207700E53E70BC053D80B8E4F53DF53EAB33AABF
:1020870034A935853E82853D83123FECFF90791454
:10209700E02532FDE43531CD253ECD353DFC740BD1
:1020A7002DF58274573CF583EFF0053EE53E70024F
:1020B700053D6420453D70C5E4FCFD9056A0E0F861
:1020C700A3E0F9A3E0FAA3E0253AFFEA3539FEEDEC
:1020D70039FDEC38FC755B01755C01755D57755E04
:1020E7000B12692FEF7002FF229079137401F080B1
:1020F7000E7420253CF53CE4353BF53B021EFD9074
:102107007913E064016056E4FFFEFDFCAB32AA31AF
:10211700A930A82FC31241D16038907915E0640126
:102127007030FCFD9056A0E0F8A3E0F9A3E0FAA315
:10213700E0253AFFEA3539FEED39FDEC38FC755BF1
:1021470001755C01755D57755E0B12692FEF7002A3
:10215700FF22053AE53A70020539021EAD90791360
:10216700E06401700302228E907934E0FCA3E0FD65
:10217700A3E0FEA3E0FF12618A90793412423D90FA
:102187005702E0FCA3E0FDA3E0FEA3E0FF90793453
:10219700E0F8A3E0F9A3E0FAA3E0FBD31241D150A2
:1021A70003022269AF48AE47AD46AC4512561590BB
:1021B700793412423DE4FFFEFDFC907934E0F8A348
:1021C700E0F9A3E0FAA3E0FBC31241D17002FF22BA
:1021D700907934E0FCA3E0FDA3E0FEA3E0FF1267E3
:1021E700A89056A012423DE4F53BF53CD39056D754
:1021F700E0953C9056D6E0953B4018740B253CF58E
:10220700827457353BF583E4F0053CE53C70DD050A
:102217003B80D9E4F539F53A9056D8E0FFC3E53A63
:102227009FE5399400503BE4FCFD9056A0E0F8A3ED
:10223700E0F9A3E0FAA3E0253AFFEA3539FEED39E4
:10224700FDEC38FC755B01755C01755D57755E0BC0
:1022570012692FEF7002FF22053AE53A70BA053985
:1022670080B6905702E0FCA3E0FDA3E0FEA3E0FFE9
:10227700907934E0F8A3E0F9A3E0FAA3E0FBD312E6
:1022870041D15003021E7CAF44AE43AD42AC4190F6
:10229700400512423D90400912424900000000905B
:1022A7004005E0FCA3E0FDA3E0FEA3E0FF90400DA6
:1022B70012423D904005E0FCA3E0FDA3E0FEA3E051
:1022C700FF1267A890401112423DE4904015F0A319
:1022D700F0A3F090400404F0904018124249000027
:0E22E700000090401C124249000000007F01E0
:0122F50022C6
:0E2D7A008F328E318D308C2F8B338A34893519
:102D8800E5207002FF22904004E07002FF22E490E8
:102D98004004F0754201F543F540F541E4FFFEFDBE
:102DA800FCAB32AA31A930A82FD31241D15003026B
:102DB8002FCC904015E0FEA3E0FFEF2532FBEE3567
:102DC80031FAE43530F9E4352FF89056D6E0FEA311
:102DD800E0FFE4FCFDD31241D1400C9056D6E0F55B
:102DE8003AA3E0F53B8010904016E02532F53B9081
:102DF8004015E03531F53AD3904016E09400904004
:102E080015E094005003022EC0904011E0FCA3E0AE
:102E1800FDA3E0FEA3E0FF755B01755C01755D57DE
:102E2800755E0B1268F5EF7003022EBD904015E039
:102E3800FEA3E0FFC3E53B9FF53BE53A9EF53AE488
:102E4800F53EF53FC3E53F953BE53E953A5034AB3B
:102E580033AA34A935853F82853E83123FECFF9023
:102E68004016E0253FFD904015E0353EFC740B2DE3
:102E7800F58274573CF583EFF0053FE53F70C505D3
:102E88003E80C1904011E0FCA3E0FDA3E0FEA3E07A
:102E9800FF755B01755C01755D57755E0B12692FD7
:102EA800EF7002FF22904016E0253BF0904015E0BD
:102EB800353AF080367F0022904011E0FCA3E0FD17
:102EC800A3E0FEA3E0FF755B01E5352541F9E53494
:102ED800354085335CF55D895E12692FEF7002FF1E
:102EE80022904015E53AF0A3E53BF0AE3AAF3BAB94
:102EF80007AA06C3E5329BF532E5319AF531E5308C
:102F08009400F530E52F9400F52FE53B2541F54178
:102F1800E53A3540F5409056D7E024FFFF9056D665
:102F2800E034FFFE904015E0FCA3E0FDD39FEC9E4B
:102F38005003022DA49056D6E0FEA3E0FFED9FFFBC
:102F4800EC9E904015F0A3EFF0A3E004F09056D863
:102F5800E014FF904017E0D39F4047E4F090400D05
:102F6800E0FCA3E0FDA3E0FEA3E0FF1256159040AD
:102F78000D12423DE4FFFEFDFC90400DE0F8A3E099
:102F8800F9A3E0FAA3E0FBC31241D17002FF22903B
:102F9800400DE0FCA3E0FDA3E0FEA3E0FF1267A85C
:102FA8008019904011E0FCA3E0FDA3E0FEA3E0241B
:102FB80001FFE43EFEE43DFDE43CFC90401112427A
:102FC8003D022DA4904018E0F8A3E0F9A3E0FAA38D
:102FD800E0FBE4FCFDEB2541FFEA3540FEED39FD61
:102FE800EC38FC90401812423DE54264016003024F
:102FF8003286907930E0FCA3E0FDA3E0FEA3E0FF79
:10300800A312423D907934E0FCA3E0FDA3E0FEA3C7
:10301800E0FF1267A89056A012423DE4F53CF53D4A
:103028009056D8E0FFC3E53D9FE53C94004003027D
:10303800321FE4FCFD9056A0E0F8A3E0F9A3E0FA03
:10304800A3E0253DFFEA353CFEED39FDEC38FC7583
:103058005B01755C01755D57755E0B1268F5EF7065
:1030680002FF22E4F53EF53FD39056D7E0953F9016
:1030780056D6E0953E500302320E7425253FF58260
:103088007457353EF583E0FFE4FCFDFEC007742667
:10309800253FF5827457353EF583E0FFE48F5CF5F4
:1030A8005BF55AF559741F253FF5827457353EF57F
:1030B80083E0FFE48F60F55FF55EF55D7420253FE2
:1030C800F5827457353EF583E0FFE48F64F563F5C8
:1030D80062F561D0071265618F398E388D378C366D
:1030E800904005E0FCA3E0FDA3E0FEA3E0FFAB39C0
:1030F800AA38A937A836C31241D160030232007436
:103108000B253FF5827457353EF583E064E570037F
:10311800023200904009E0FCA3E0FDA3E0FEA3E03A
:10312800FF904018E0F8A3E0F9A3E0FAA3E0FBD38E
:103138001241D14014904018E0FCA3E0FDA3E0FE4A
:10314800A3E0FF90400912423D904009A3A3A3E0E9
:10315800FF7427253FF5827457353EF583EFF090CD
:103168004009E0FCA3E0FDA3E0FEA3E0FF7808121D
:1031780041E27428253FF5827457353EF583EFF018
:10318800904009E0FCA3E0FDA3E0FEA3E0FF781077
:103198001241E27429253FF5827457353EF583EFD5
:1031A800F0904009E0FCA3E0FDA3E0FEA3E0FF7877
:1031B800181241E2742A253FF5827457353EF5838B
:1031C800EFF0E4FCFD9056A0E0F8A3E0F9A3E0FAE4
:1031D800A3E0253DFFEA353CFEED39FDEC38FC75F2
:1031E8005B01755C01755D57755E0B12692FEF7099
:1031F80002FF22754301800E7420253FF53FE43518
:103208003EF53E023070E5436401600B053DE53D47
:103218007002053C023028E5436401603C90793433
:10322800E0FCA3E0FDA3E0FEA3E0FF12618A907931
:103238003412423D905702E0FCA3E0FDA3E0FEA358
:10324800E0FF907934E0F8A3E0F9A3E0FAA3E0FB0B
:10325800D31241D1500302300C905702E0FCA3E096
:10326800FDA3E0FEA3E0FF907934E0F8A3E0F9A322
:10327800E0FAA3E0FBD31241D140037F0022904043
:05328800047401F0FFD9
:01328D00221E
:064A58008B2F8A3089312A
:104A5E00E5207002FF22907930E0FCA3E0FDA3E098
:104A6E00FEA3E0FFA312423D907934E0FCA3E0FDEB
:104A7E00A3E0FEA3E0FF1267A89056A012423DE409
:104A8E00F532F5339056D8E0FFC3E5339FE5329407
:104A9E00004003024C5BE4FCFD9056A0E0F8A3E05E
:104AAE00F9A3E0FAA3E02533FFEA3532FEED39FD36
:104ABE00EC38FC755B01755C01755D57755E0B120C
:104ACE0068F5EF7002FF22E4F534F535D39056D732
:104ADE00E095359056D6E095345003024C4A740B4F
:104AEE002535F58274573534F583E07002FF22E4E4
:104AFE00F537AB2FAA30A931853782758300123F67
:104B0E00ECFFE5377C002535FDEC3534FC740B2DC0
:104B1E00F58274573CF583E0B507090537E537D3C1
:104B2E00940A40CEE537D3940A5003024C3C740BE2
:104B3E002535F58274573534F58374E5F0742525E3
:104B4E0035F58274573534F583E0FFE4FCFDFEC085
:104B5E000774262535F58274573534F583E0FFE466
:104B6E008F5CF55BF55AF559741F2535F582745730
:104B7E003534F583E0FFE48F60F55FF55EF55D7427
:104B8E00202535F58274573534F583E0FFE48F64C4
:104B9E00F563F562F561D00712656190400512422A
:104BAE003DE53524E0FFE53434FFFEC3EE6480942A
:104BBE0080402574162FF58274573EF583E0B40FAE
:104BCE0017740B2FF58274573EF58374E5F074E07D
:104BDE002FFF74FF3EFE80D37F0F126A68E4FCFD48
:104BEE009056A0E0F8A3E0F9A3E0FAA3E02533FF86
:104BFE00EA3532FEED39FDEC38FC755B01755C0172
:104C0E00755D57755E0B12692FEF7002FF227F0ADA
:104C1E00126A68904005E0FCA3E0FDA3E0FEA3E06D
:104C2E00FF125307EF7002FF22753601800E7420BB
:104C3E002535F535E43534F534024ADAE5366401C6
:104C4E00600B0533E53370020532024A92E5366495
:104C5E0001603C907934E0FCA3E0FDA3E0FEA3E00C
:104C6E00FF12618A90793412423D905702E0FCA304
:104C7E00E0FDA3E0FEA3E0FF907934E0F8A3E0F9B5
:104C8E00A3E0FAA3E0FBD31241D15003024A76907F
:104C9E005702E0FCA3E0FDA3E0FEA3E0FF90793411
:104CAE00E0F8A3E0F9A3E0FAA3E0FBD31241D14070
:064CBE00037F00227F01CC
:014CC40022CD
:10577600E5207002FF229056EEA3A3E0FEA3E08E82
:105786002FF530E4F538F537F536F5359056EEE079
:10579600FCA3E0FDA3E0FEA3E0FF9056FAE0F8A329
:1057A600E0F9A3E0FAA3E02FFBEA3EFAE93DF9E8C7
:1057B6003CF8AE2FAF30E4FCFDD31241D1500302CA
:1057C6005862AE2FAF30E4FCFD755B01755C017568
:1057D6005D57755E0B1268F5EF6070E4FBFAD390C7
:1057E60056D7E09B9056D6E09A4063740B2BF58211
:1057F60074573AF583E07027740C2BF58274573A88
:10580600F583E0701A740D2BF58274573AF583E030
:10581600700D740E2BF58274573AF583E060067EA0
:10582600007F0180047E007F00EF4E7015E538246E
:1058360001F538E43537F537E43536F536E43535F0
:10584600F53574042BFBE43AFA80937F0022053089
:10585600E5306003025792052F0257929056D8E022
:10586600FF7E009056D6E0FCA3E0FD12404DE48F8B
:10587600348E33F532F531AD32AC31AB38AA37A9B7
:1058860036A8351240B48F348E338D328C31781869
:105896001241E2900002EFF0AF34AE33AD32AC31DC
:1058A60078101241E2A3EFF0AF34AE33AD32AC3133
:1058B60078081241E2A3EFF0E534FFA3EFF090562B
:0A58C600CA124249000000047F01ED
:0158D00022B5
:0E1057008F328E318D308C2F8B338A34893559
:10106500E5207002FF22E532541FFFE4FEFDFCFB84
:10107500FAF9F8C31241D160037F0022E53224203A
:10108500FBE43531FAE43530F9E4352FF89056D6DE
:10109500E0FEA3E0FFE4FCFDD31241D140037F0055
:1010A50022E4904004F090401C12424900000000E8
:1010B5001239908F448E438D428C41E47F02FEFDB0
:1010C500FCAB44AA43A942A841C31241D150037FB6
:1010D5000022AB33AA34A93590000B741012402BB3
:1010E500AF44AE43AD42AC4178181241E2900015D1
:1010F500EF12402BAF44AE43AD42AC4178101241E4
:10110500E2900014EF12402BAF44AE43AD42AC4128
:1011150078081241E290001BEF12402B90001AE56F
:101125004412402B90001CE412402B90001DE41249
:10113500402B90001EE412402B90001FE412402B20
:10114500E4907913F0907930E0FCA3E0FDA3E0FE94
:10115500A3E0FFA312423D907934E0FCA3E0FDA398
:10116500E0FEA3E0FF1267A89056A012423D9079D9
:1011750034E0FCA3E0FDA3E0FEA3E0F5488E478D37
:10118500468C45E4F539F53A9056D8E0FFC3E53A83
:101195009FE53994004003021444E4FCFD9056A0F9
:1011A500E0F8A3E0F9A3E0FAA3E0253AFFEA353930
:1011B500FEED39FDEC38FC755B01755C01755D571D
:1011C500755E0B1268F5EF7002FF22E4F53FF540FE
:1011D500907915F0F53BF53CD39056D7E0953C90CA
:1011E50056D6E0953B50030213E6E4FFFEFDFCAB4B
:1011F50032AA31A930A82F1241D160030212877497
:101205000B253CF5827457353BF583E0600764E5B3
:1012150060030213D8E4F53DF53EAB33AA34A93596
:10122500853E82853D83123FECFFE53C253EFDE58D
:101235003B353DFC740B2DF58274573CF583EFF07F
:10124500053EE53E7002053D6420453D70CCE4FC5D
:10125500FD9056A0E0F8A3E0F9A3E0FAA3E0253A53
:10126500FFEA3539FEED39FDEC38FC755B01755C3F
:1012750001755D57755E0B12692FEF7002FF220233
:1012850013D0E540453F7006907914E53CF0740BAA
:10129500253CF5827457353BF583E0FFB4E50A0537
:1012A50040E540702B053F8027EF701F0540E54066
:1012B5007002053F740B253CF5827457353BF58369
:1012C50074E5F09079157401F08005E4F53FF5407B
:1012D500E5322420FFE43531FEE43530FDE4352FD9
:1012E500FCC004C005C006C007E540AE3F7805C395
:1012F50033CE33CED8F9FBAA06E4F9F8D007D006E9
:10130500D005D004C31241D150030213D8E4F53DF2
:10131500F53EAE3DAF3EE4FCFDAB32AA31A930A8A7
:101325002FD31241D14033AB36AA37A938853E8237
:10133500853D83123FECFF907914E07C00253EFD4E
:10134500EC353DFC740B2DF58274573CF583EFF0BD
:10135500053EE53E70BC053D80B8E4F53DF53EAB88
:1013650033AA34A935853E82853D83123FECFF9033
:101375007914E02532FDE43531CD253ECD353DFCF2
:10138500740B2DF58274573CF583EFF0053EE53E71
:101395007002053D6420453D70C5E4FCFD9056A0F6
:1013A500E0F8A3E0F9A3E0FAA3E0253AFFEA35392E
:1013B500FEED39FDEC38FC755B01755C01755D571B
:1013C500755E0B12692FEF7002FF2290791374017D
:1013D500F0800E7420253CF53CE4353BF53B0211CD
:1013E500DD907913E064016056E4FFFEFDFCAB324D
:1013F500AA31A930A82FC31241D16038907915E0E0
:1014050064017030FCFD9056A0E0F8A3E0F9A3E07C
:10141500FAA3E0253AFFEA3539FEED39FDEC38FC53
:10142500755B01755C01755D57755E0B12692FEF74
:101435007002FF22053AE53A7002053902118D90D6
:101445007913E06401700302156E907934E0FCA312
:10145500E0FDA3E0FEA3E0FF12618A907934124219
:101465003D905702E0FCA3E0FDA3E0FEA3E0FF9062
:101475007934E0F8A3E0F9A3E0FAA3E0FBD3124145
:10148500D15003021549AF48AE47AD46AC4512569B
:101495001590793412423DE4FFFEFDFC907934E06D
:1014A500F8A3E0F9A3E0FAA3E0FBC31241D170026F
:1014B500FF22907934E0FCA3E0FDA3E0FEA3E0FF6A
:1014C5001267A89056A012423DE4F53BF53CD39037
:1014D50056D7E0953C9056D6E0953B4018740B25C1
:1014E5003CF5827457353BF583E4F0053CE53C70EB
:1014F500DD053B80D9E4F539F53A9056D8E0FFC3D0
:10150500E53A9FE5399400503BE4FCFD9056A0E098
:10151500F8A3E0F9A3E0FAA3E0253AFFEA3539FE9E
:10152500ED39FDEC38FC755B01755C01755D577532
:101535005E0B12692FEF7002FF22053AE53A70BA89
:10154500053980B6905702E0FCA3E0FDA3E0FEA3B9
:10155500E0FF907934E0F8A3E0F9A3E0FAA3E0FB1B
:10156500D31241D1500302115C905702E0FCA3E075
:10157500FDA3E0FEA3E0FF907934E0F8A3E0F9A332
:10158500E0FAA3E0FBD31241D140037F0022753B73
:1015950000753C40D39056D7E0953C9056D6E095E3
:1015A5003B4018740B253CF5827457353BF583E4B5
:1015B500F0053CE53C70DD053B80D9E4F53BF53CA9
:1015C500740B253CF5827457353BF5837420F00583
:1015D5003CE53C7002053B642B453B70E390570BA3
:1015E500742EF0753B00753C0BAB33AA34A93585D9
:1015F5003C82853B83123FECFF740B253CF58274DE
:1016050057353BF583EFF0053CE53C7002053B643F
:1016150020453B70D490572B742EF0A3F0753B00FA
:10162500753C2BAB33AA34A935E53C24E0FFE53BFB
:1016350034FF8F82F583123FECFF740B253CF58256
:101645007457353BF583EFF0053CE53C7002053BEF
:101655006440453B70CD9056FEE0FCA3E0FDA3E061
:10166500FEA3E0FF907930E0F8A3E0F9A3E0FAA348
:10167500E0FBC31241D1700E905740F090573FF0F8
:10168500905746F0804F907930E0FCA3E0FDA3E051
:10169500FEA3E0FF78181241E2905740EFF09079F1
:1016A50030E0FCA3E0FDA3E0FEA3E0FF78101241CB
:1016B500E290573FEFF0907930E0FCA3E0FDA3E026
:1016C500FEA3E0FF78081241E2905746EFF09079CB
:1016D50030A3A3A3E0905745F0AF44AE43AD42AC71
:1016E500411267A89056A012423D9056A0E0FCA377
:1016F500E0FDA3E0FEA3E0FF755B01755C01755D90
:1017050057755E0B12692FEF7002FF22AF44AE438F
:10171500AD42AC4190793012423D90400D124249A4
:06172500000000007F013E
:01172B00229B
:06511D007B017A5679A91E
:065123008B2F8A30893158
:10512900E5207002FF22E4904004F0F535907930D3
:10513900E0FCA3E0FDA3E0FEA3E0FFA312423D9043
:105149007934E0FCA3E0FDA3E0FEA3E0FF1267A829
:105159009056A012423DE4F5369056D8E0FFE53668
:10516900C39F400302522FE4FCFDFE9056A0E0F8D5
:10517900A3E0F9A3E0FAA3E02536FFEE3AFEED3904
:10518900FDEC38FC755B01755C01755D57755E0B4F
:105199001268F5EF7002FF22E4F532F533D3905629
:1051A900D7E095339056D6E09532406F740B25338E
:1051B900F58274573532F583E07002FF22E4F53445
:1051C900AB2FAA30A931853482758300123FECFFD9
:1051D900E5347C002533FDEC3532FC740B2DF5826A
:1051E90074573CF583E0B507090534E534D3940ACF
:1051F90040CEE534D3940A401574162533F58274EC
:10520900573532F583E030E405753501800D74209A
:105219002533F533E43532F5328082E535640160B2
:10522900050536025162E5356401603C907934E048
:10523900FCA3E0FDA3E0FEA3E0FF12618A907934AC
:1052490012423D905702E0FCA3E0FDA3E0FEA3E07B
:10525900FF907934E0F8A3E0F9A3E0FAA3E0FBD3E7
:105269001241D15003025148905702E0FCA3E0FDDE
:10527900A3E0FEA3E0FF907934E0F8A3E0F9A3E00E
:10528900FAA3E0FBD31241D140037F002274252504
:1052990033F58274573532F583E0FFE4FCFDFEC037
:1052A9000774262533F58274573532F583E0FFE418
:1052B9008F5CF55BF55AF559741F2533F5827457E0
:1052C9003532F583E0FFE48F60F55FF55EF55D74D7
:1052D900202533F58274573532F583E0FFE48F6476
:1052E900F563F562F561D007126561907930124274
:0D52F9003D90400D124249000000007F0171
:015306002284
:10609A00E5207002FF229056FEE0FCA3E0FDA3E09B
:1060AA00FEA3E0FF907930E0F8A3E0F9A3E0FAA3B9
:1060BA00E0FBC31241D170037F0122E4904004F057
:1060CA00907930E0FCA3E0FDA3E0FEA3E0FF1267B5
:1060DA00A89056A012423D9056A0E0FCA3E0FDA372
:1060EA00E0FEA3E0FF755B01755C01755D57755EA7
:1060FA000B1268F5EF7002FF2290572BE0642E60B6
:10610A0009A3E0642E60037F0022905745E0FFE474
:10611A00FCFDFEC007A3E0FFE48F5CF55BF55AF5D2
:10612A005990573FE0FFE48F60F55FF55EF55DA398
:10613A00E0FFE48F64F563F562F561D007126561EB
:10614A0090793012423DE4FFFEFDFC907930E0F890
:10615A00A3E0F9A3E0FAA3E0FBC31241D1701490C3
:10616A0056FEE0FCA3E0FDA3E0FEA3E0FF90793039
:10617A0012423D90400D124249000000007F012268
:10698C00E5207002FF22E4904004F09056FEE0FCFB
:10699C00A3E0FDA3E0FEA3E0FF90793012423D7F1F
:0269AC000122C6
:0867A8008F4C8E4B8D4A8C4989
:1067B000E54C24FEF550E54B34FFF54FE54A34FF38
:1067C000F54EE54934FFF54D9056D8E0FFE4FCFD69
:1067D000FEAB50AA4FA94EA84D1240B48F508E4F19
:1067E0008D4E8C4D9056F6E0FCA3E0FDA3E0FEA399
:1067F000E02550F550EE354FF54FED354EF54EECAA
:0B680000354DF54DAF50AE4FAD4EFCD6
:01680B00226A
:08680C008F588E578D568C55F4
:106814009056D6E0FEA3E07802CEC313CE13D8F987
:10682400FBAA06E4F9F8AF58AE57AD56AC55124181
:106834003F8F5C8E5B8D5A8C599056EEE0FCA3E042
:10684400FDA3E0FEA3E0255CF55CEE355BF55BEDB6
:10685400355AF55AEC3559F559AF5CAE5BAD5AFC77
:016864002211
:1068BA008F588E578D568C559056D6E0FEA3E078A9
:1068CA0002CEC313CE13D8F9FBAA06E4F9F8AF58DF
:1068DA00AE57AD56AC5512413FAC00AD01AE02AF5A
:0B68EA0003E47B04FAF9F81240B4222A
:08618A008F4C8E4B8D4A8C49AD
:1061920012680C8F508E4F8D4E8C4DAF4CAE4BAD66
:1061A2004AAC491268BA8F548E538D528C51AF50FB
:1061B200AE4FAD4EAC4D90401CE0F8A3E0F9A3E029
:1061C200FAA3E0FBC31241D1602FAF50AE4FAD4EE8
:1061D200AC4D755B01755C01755D77755E0B126880
:1061E200F5EF700774FFFFFEFDFC22AF50AE4FAD1E
:1061F2004EAC4D90401C12423D740B2554F58274F6
:10620200773553F583E0FFE4FCFDFEC007AA53ABEC
:1062120054740C2BF58274773AF583E0FFE48F5CBB
:10622200F55BF55AF559740D2BF58274773AF583BF
:10623200E0FFE48F60F55FF55EF55D740E2554F5C1
:106242008274773553F583E0FFE48F64F563F5627A
:0F625200F561D0071265618F4C8E4B8D4A8C49D8
:01626100221A
:085C4A008F368E358D348C334A
:105C52009056D8E0FF7E009056D6E0FCA3E0FD12FD
:105C6200404D8E378F38904005E0FCA3E0FDA3E065
:105C7200FEA3E0FF90400D12423DAE37AF38E4FC88
:105C8200FDAB36AA35A934A833D31241D14051AE67
:105C920037AF38AB07AA06E5369BF536E5359AF5F8
:105CA20035E5349400F534E5339400F53390400D36
:105CB200E0FCA3E0FDA3E0FEA3E0FF12618A9040B6
:105CC2000D12423D74FFFFFEFDFC90400DE0F8A373
:105CD200E0F9A3E0FAA3E0FBC31241D1709CFF22DA
:105CE2009056D6E0FEA3E0FBAA06E4F9F8AF36AE82
:105CF20035AD34AC3312413F904017EFF090400D78
:105D0200E0FCA3E0FDA3E0FEA3E0FF1267A8A80465
:105D1200A905AA06AB07904017E0FFE4FCFDFEEBE5
:105D22002FFFEE3AFEED39FDEC38FC9040111242A5
:105D32003D9056D6E0FEA3E0FBAA06E4F9F8AF36A2
:105D4200AE35AD34AC3312413FAF03904015EAF0AB
:0F5D5200A3EFF090401C124249000000007F01B7
:015D6100221F
:085307008F3B8E3A8D398C3882
:10530F00E47F01FEFDFCAB3BAA3AA939A838D312C2
:10531F0041D1500302549E905702E0FCA3E0FDA33D
:10532F00E0FEA3E0FFA8381241D1400302549EAF24
:10533F003BAE3AAD39AC3812680C8F3F8E3E8D3D87
:10534F008C3CAF3BAE3AAD39AC381268BA8F438E56
:10535F00428D418C40AF3FAE3EAD3DAC3C755B01E5
:10536F00755C01755D57755E0B1268F5EF70030282
:10537F005413905706E0FCA3E0FDA3E0FEA3E0FF6B
:10538F00AB3BAA3AA939A838C31241D1500EAF3B53
:10539F00AE3AAD39AC3890570612423D740B2543E7
:1053AF00F58274573542F583E0FFE4FCFDFEC0073C
:1053BF00AA42AB43740C2BF58274573AF583E0FF86
:1053CF00E48F5CF55BF55AF559740D2BF582745724
:1053DF003AF583E0FFE48F60F55FF55EF55D740EDF
:1053EF002543F58274573542F583E0FFE48F64F56A
:1053FF0063F562F561D0071265618F3B8E3A8D3987
:10540F008C3880037F0022AE42AF43740B2FF5829E
:10541F0074573EF583E4F0740C2FF58274573EF504
:10542F0083E4F0740D2FF58274573EF583E4F07426
:10543F000E2FF58274573EF583E4F0F5449056D95C
:10544F00E0FFE544C39F400302530F7F05126A68D4
:10545F00AF44E4FCFDFE9056FAE0F8A3E0F9A3E0B8
:10546F00FAA3E0FB1240B4EF253FFFEE353EFEED11
:10547F00353DFDEC353CFC755B01755C01755D5789
:10548F00755E0B12692FEF7002FF22054480AE7F0D
:01549F00010B
:0154A00022E9
:10399000905706E0FCA3E0FDA3E0FEA3E0FF126861
:1039A0000C90792B12423D9056EEE0F8A3E0F9A37B
:1039B000E0FAA3E0FB90792BE0FCA3E0FDA3E0FE9E
:1039C000A3E0C39BFFEE9AFEED99FDEC98FCC004CA
:1039D000C005C006C0079056D6E0FEA3E07802CE30
:1039E000C313CE13D8F9FFE4FCFDD003D002D001FD
:1039F000D0001240B490792312423D9056EEE0FC84
:103A0000A3E0FDA3E0FEA3E0FF9056FAE0F8A3E0F8
:103A1000F9A3E0FAA3E02FFFEA3EFEE93DFDE83C12
:103A2000FC90792BE0F8A3E0F9A3E0FAA3E0FBC354
:103A30001241D14003023CC190792BE0FCA3E0FD90
:103A4000A3E0FEA3E0FF755B01755C01755D577532
:103A50005E0B1268F5EF7003023CC29079271242A8
:103A600049000000009056D6E0FEA3E0FFE4FCFD14
:103A7000907927E0F8A3E0F9A3E0FAA3E0FBC312F2
:103A800041D14003023C56907927A3A3E0FEA3E076
:103A9000FF240BF58274573EF583E06003023C344B
:103AA000740C2FF58274573EF583E06003023C34BA
:103AB000907927A3A3A3E0240DF58274573EF583E4
:103AC000E06003023C34740E2FF58274573EF58398
:103AD000E06003023C34907927A3A3A3E0240BF514
:103AE0008274573EF58374FFF0740C2FF58274577F
:103AF0003EF58374FFF0740D2FF58274573EF58305
:103B000074FFF0740E2FF58274573EF58374FFF046
:103B1000E490792FF09056D9E0FF90792FE0C39F81
:103B200050547F05126A6890792FE0FFE4FCFDFE97
:103B30009056FAE0F8A3E0F9A3E0FAA3E0FB124004
:103B4000B490792BE0F8A3E0F9A3E0FAA3E02FFF0B
:103B5000EA3EFEE93DFDE83CFC755B01755C0175E4
:103B60005D57755E0B12692FEF7003023CC29079AE
:103B70002FE004F0809F907923E0F8A3E0F9A3E020
:103B8000FAA3E0FBC000C001C002C003E47B04FA5A
:103B9000F9F8A3E0FCA3E0FDA3E0FEA3E0FF1241DF
:103BA0003FD003D002D001D000EB2FFFEA3EFEE968
:103BB0003DFDE83CFC90792312423D907923E0FCE6
:103BC000A3E0FDA3E0FEA3E024FEFFEE34FFFEED44
:103BD00034FFFDEC34FFFC905702E0F8A3E0F9A3BA
:103BE000E0FAA3E0FBD31241D14045905706E0FC38
:103BF000A3E0FDA3E0FEA3E0FF907923E0F8A3E0BB
:103C0000F9A3E0FAA3E0FBD31241D1401490792349
:103C1000E0FCA3E0FDA3E0FEA3E0FF905706124204
:103C20003D907923E0FCA3E0FDA3E0FEA3E0FF22AA
:103C3000E4023CC2907927E0FCA3E0FDA3E0FEA3F0
:103C4000E02404FFE43EFEE43DFDE43CFC907927E3
:103C500012423D023A65907923E0F8A3E0F9A3E02F
:103C6000FAA3E0FBC000C001C002C0039056D6E03A
:103C7000FEA3E07802CEC313CE13D8F9FFE4FCFD17
:103C8000D003D002D001D000EB2FFFEA3EFEED3989
:103C9000FDEC38FC90792312423D90792BE0FCA397
:103CA000E0FDA3E0FEA3E02401FFE43EFEE43DFDD1
:103CB000E43CFC90792B12423D7F01126A68023984
:063CC000FBE4FFFEFDFC29
:013CC60022DB
:085615008F4C8E4B8D4A8C492D
:10561D0012399090791612423DAF4CAE4BAD4AAC5B
:10562D004912680C90791A12423DAF4CAE4BAD4AFF
:10563D00AC491268BA90791E12423D90791AE0FC7D
:10564D00A3E0FDA3E0FEA3E0FF755B01755C0175B2
:10565D005D57755E0B1268F5EF7003025761907917
:10566D0016A3A3A3E0FB90791EA3A3E0FEA3E02461
:10567D000BF58274573EF583EBF0907916E0FCA3A1
:10568D00E0FDA3E0FEA3E0FF78081241E290791E51
:10569D00A3A3E0FEA3E0240CF58274573EF583EF3F
:1056AD00F0907916E0FCA3E0FDA3E0FEA3E0FF7807
:1056BD00101241E290791EA3A3E0FEA3E0240DF5A4
:1056CD008274573EF583EFF0907916E0FCA3E0FD70
:1056DD00A3E0FEA3E0FF78181241E290791EA3A388
:1056ED00E0FEA3E0240EF58274573EF583EFF0E45F
:1056FD00907922F09056D9E0FF907922E0C39F5027
:10570D00597F05126A68907922E0FFE4FCFDFE9056
:10571D0056FAE0F8A3E0F9A3E0FAA3E0FB1240B4D7
:10572D0090791AE0F8A3E0F9A3E0FAA3E02FFFEADD
:10573D003EFEE93DFDE83CFC755B01755C01755D68
:10574D0057755E0B12692FEF70028009907922E078
:10575D0004F080A0E4FFFEFDFC22907916E0FCA38E
:08576D00E0FDA3E0FEA3E0FF54
:015775002211
:10284F009056D67402F0A3E4F0755B01755C0175C8
:10285F005D57755E0BFFFEFDFC1268F5EF7002FF12
:10286F0022905909E0B45506A3E064AA60037F00E3
:10287F002290570BE064EB6004E0B4E90C9056CE65
:10288F001242490000000080489058C9E0648060FF
:10289F0006E060037F00229058D1E0FFE4FCFDFECC
:1028AF00C007A3E0FFE48F5CF55BF55AF559A3E091
:1028BF00FFE48F60F55FF55EF55DA3E0FFE48F64E5
:1028CF00F563F562F561D0071265619056CE12423D
:1028DF003D9056CEE0FCA3E0FDA3E0FEA3E0FF7524
:1028EF005B01755C01755D57755E0B1268F5EF70D6
:1028FF0002FF22905909E0B45506A3E064AA6003D1
:10290F007F0022905716E0FF7E00A3E0FD7C0012AF
:10291F006A389056D6EEF0A3EFF0905718E0905625
:10292F00D8F0905719E0FF7E00A3E0FD7C00126AFB
:10293F00388E2F8F3090571BE09056D9F090575DFF
:10294F00E064466003022B69A3E064416003022B3D
:10295F0069A3E064546003022B69A3E0643360034E
:10296F00022B69A3E064326003022B6990571CE0CD
:10297F00FF7E00A3E0FD7C00126A389056DAEEF07D
:10298F00A3EFF09056DAE0FEA3E07805C333CE3321
:10299F00CED8F9FF9056D6E0FCA3E0FD12405F9031
:1029AF0056DAEEF0A3EFF090572BE0FFE4FCFDFEBC
:1029BF00C007A3E0FFE48F5CF55BF55AF559A3E080
:1029CF00FFE48F60F55FF55EF55DA3E0FFE48F64D4
:1029DF00F563F562F561D0071265619056EA124210
:1029EF003D90572FE0FFE4FCFDFEC007A3E0FFE49E
:1029FF008F5CF55BF55AF559A3E0FFE48F60F55F47
:102A0F00F55EF55DA3E0FFE48F64F563F562F561B4
:102A1F00D0071265619056FA12423D905737E0FF8A
:102A2F00E4FCFDFEC007A3E0FFE48F5CF55BF55A05
:102A3F00F559A3E0FFE48F60F55FF55EF55DA3E068
:102A4F00FFE48F64F563F562F561D007126561905D
:102A5F0056FE12423DE4FCFD9056CEE0F8A3E0F99D
:102A6F00A3E0FAA3E02530FFEA352FFEED39FDECA8
:102A7F0038FC9056EE12423D9056D9E0FFE4FCFD33
:102A8F00FE9056FAE0F8A3E0F9A3E0FAA3E0FB12F8
:102A9F0040B49056EEE0F8A3E0F9A3E0FAA3E02FDC
:102AAF00FFEA3EFEE93DFDE83CFC9056F612423D42
:102ABF009056D9E0FFE4FCFDFE9056FAE0F8A3E053
:102ACF00F9A3E0FAA3E0FB1240B4A804A905C006DD
:102ADF00C007AE2FAF30AB07AA069056EAE0FCA3B3
:102AEF00E0FDA3E0FEA3E0C39BFFEE9AFEED940092
:102AFF00FDEC9400FCD003D002C3EF9BFFEE9AFED7
:102B0F00ED99FDEC98FCC006C0079056DAE0FEA3E5
:102B1F00E0FBAA06D007D006C3EF9BFFEE9AFEEDAF
:102B2F009400FDEC9400FCC0079056D8E0FBE4FA4B
:102B3F00F9F8D00712413F90570212423D9056FECE
:102B4F00E0FCA3E0FDA3E0FEA3E0FF90793012428A
:102B5F003D90570A7401F0022D7290571CE0FF7ED2
:102B6F0000A3E0FD7C00126A389056DAEEF0A3EF76
:102B7F00F09056DAE0FEA3E07805C333CE33CED81B
:102B8F00F9FF9056D6E0FCA3E0FD12405F9056DAB5
:102B9F00EEF0A3EFF090571EE0FF7E00A3E0FD7C68
:102BAF0000126A38E4FCFD9056DC12423DE4FFFE51
:102BBF00FDFC9056DCE0F8A3E0F9A3E0FAA3E0FBFC
:102BCF00C31241D1703A90572BE0FFE4FCFDFEC0D9
:102BDF0007A3E0FFE48F5CF55BF55AF559A3E0FF1F
:102BEF00E48F60F55FF55EF55DA3E0FFE48F64F5BC
:102BFF0063F562F561D0071265619056DC12423DB4
:102C0F00905721E0FF7E00A3E0FD7C00126A389010
:102C1F0056E0EEF0A3EFF0E4FCFD9056CEE0F8A303
:102C2F00E0F9A3E0FAA3E02530FFEA352FFEED39F6
:102C3F00FDEC38FC9056EE12423D9056D9E0FF7EE7
:102C4F00009056E0E0FCA3E0FD12404DE4FCFD9047
:102C5F0056CEE0F8A3E0F9A3E0FAA3E02FFBEA3E9B
:102C6F00FAED39F9EC38F8EB2530FFEA352FFEEDA8
:102C7F0039FDEC38FC9056F212423D9056D9E0FFE8
:102C8F007E009056E0E0FCA3E0FD12404DE4FCFD19
:102C9F009056EEE0F8A3E0F9A3E0FAA3E02FFBEAE9
:102CAF003EFAED39F9EC38F89056DAE0FEA3E0FF82
:102CBF00EB2FFFEA3EFEED39FDEC38FC9056F61295
:102CCF00423D9056DAE0FEA3E0FBAA06A3E0FCA388
:102CDF00E0FDA3E0FEA3E0C39BFFEE9AFEED9400A0
:102CEF00FDEC9400FCC004C005C006C0079056D987
:102CFF00E0FF7E009056E0E0FCA3E0FD12404DABFC
:102D0F0007AA06D007D006D005D004C3EF9BFFEE6D
:102D1F009AFEED9400FDEC9400FCEF24FFFFEE34DF
:102D2F00FFFEED34FFFDEC34FFFCC0079056D8E0FA
:102D3F00FBE4FAF9F8D00712413F90570212423DD7
:102D4F00E47FF57E0FFDFC905702E0F8A3E0F9A3B6
:102D5F00E0FAA3E0FBC31241D150037F0022E490BD
:0A2D6F00570AF0E4904004F07F01E1
:012D79002237
:1068F5008F5A8E598D588C57AF5B155BEF6028AB5F
:106905005CAA5DA95EAF5AAE59AD58AC577809126D
:1069150041F51264DCEF7002FF22E4255EF55E743A
:0A69250002355DF55D80D17F01228F
:10692F008F5A8E598D588C57AF5B155BEF6028AB24
:10693F005CAA5DA95EAF5AAE59AD58AC5778091233
:10694F0041F5126314EF7002FF22E4255EF55E74C9
:0A695F0002355DF55D80D17F012255
:03000000026A543D
:0C6A5400787FE4F6D8FD75816B025D626E
:103FD300BB010689828A83E0225002E722BBFE02EC
:093FE300E32289828A83E493221F
:103FEC00BB010CE58229F582E5833AF583E022508A
:103FFC0006E92582F8E622BBFE06E92582F8E222D4
:0D400C00E58229F582E5833AF583E49322ED
:10401900BB010689828A83F0225002F722BBFE0186
:02402900F32280
:10402B00F8BB010DE58229F582E5833AF583E8F0CB
:10403B00225006E92582C8F622BBFE05E92582C877
:02404B00F2225F
:10404D00EF8DF0A4A8F0CF8CF0A428CE8DF0A42E87
:02405D00FE2241
:10405F00BC000BBE0029EF8DF084FFADF022E4CC45
:10406F00F875F008EF2FFFEE33FEEC33FCEE9DEC0E
:10407F00984005FCEE9DFE0FD5F0E9E4CEFD22ED54
:10408F00F8F5F0EE8420D21CFEADF075F008EF2F9E
:10409F00FFED33FD4007985006D5F0F222C398FD8F
:0540AF000FD5F0EA222C
:1040B400E88FF0A4CC8BF0A42CFCE98EF0A42CFCAB
:1040C4008AF0EDA42CFCEA8EF0A4CDA8F08BF0A429
:1040D4002DCC3825F0FDE98FF0A42CCD35F0FCEB88
:1040E4008EF0A4FEA9F0EB8FF0A4CFC5F02ECD394D
:0F40F400FEE43CFCEAA42DCE35F0FDE43CFC22BA
:1041030075F008758200EF2FFFEE33FECD33CDCC73
:1041130033CCC58233C5829BED9AEC99E5829840F6
:104123000CF582EE9BFEED9AFDEC99FC0FD5F0D6D3
:10413300E4CEFBE4CDFAE4CCF9A88222B800C1B9FD
:104143000059BA002DEC8BF084CFCECDFCE5F0CB3B
:10415300F97818EF2FFFEE33FEED33FDEC33FCEB74
:1041630033FB10D703994004EB99FB0FD8E5E4F92F
:10417300FA227818EF2FFFEE33FEED33FDEC33FC1C
:10418300C933C910D7059BE99A4007EC9BFCE99A10
:10419300F90FD8E0E4C9FAE4CCFB2275F010EF2F55
:1041A300FFEE33FEED33FDCC33CCC833C810D70755
:1041B3009BEC9AE899400AED9BFDEC9AFCE899F890
:0E41C3000FD5F0DAE4CDFBE4CCFAE4C8F92223
:1041D100EB9FF5F0EA9E42F0E99D42F0E89C45F044
:0141E10022BB
:1041E200E8600FECC313FCED13FDEE13FEEF13FFBB
:0341F200D8F122DF
:1041F500E8600FEFC333FFEE33FEED33FDEC33FC28
:03420500D8F122CB
:104208007401FF3395E0FEFDFCA3A3A3E02FFFF0AC
:10421800E582158270021583E03EFEF0E582158284
:1042280070021583E03DFDF0E5821582700215836A
:05423800E03CFCF02257
:0C423D00ECF0A3EDF0A3EEF0A3EFF022F4
:10424900A8828583F0D083D0821242601242601224
:104259004260124260E473E493A3C583C5F0C58349
:10426900C8C582C8F0A3C583C5F0C583C8C582C8BF
:014279002222
:0C427A00A42582F582E5F03583F583224F
:00000001FF
